:0200000480007A
:10000000B72F0000938F0F8073900F306F00400365
:100010001300000013000000130000001300000094
:100020001300000013000000130000001300000084
:100030001300000013000000130000001300000074
:100040009702000093824211739052309300000097
:10005000130100009301000013020000930200004E
:100060001303000093030000130400009304000036
:10007000130500009305000013060000930600001E
:100080001307000093070000130800009308000006
:100090001309000093090000130A0000930A0000EE
:1000A000130B0000930B0000130C0000930C0000D6
:1000B000130D0000930D0000130E0000930E0000BE
:1000C000130F0000930F0000971102009381C1C12C
:1000D00017050200130505439795030093854571A5
:1000E00013060000EF00001A170502001305C536BD
:1000F000970502009385053F13060000EF00801866
:1001000017A503001305056F97B503009385456E8A
:1001100037B6ABAB1306B6BAEF00C01617B1030083
:100120001301416DEF80901F9392120093D2120041
:100130009382D2FF638A02008322010013014100EF
:100140006F0000177300203083220100130141006B
:10015000730020301301C1FF23205100F32220340B
:10016000E3C402FC8322010013014100130141F8A2
:1001700023221100232421002326310023284100BB
:10018000232A5100232C6100232E71002320810299
:10019000232291022324A1022326B1022328C10293
:1001A000232AD102232CE102232EF1022320010570
:1001B0002322110523242105232631052328410567
:1001C000232A5105232C6105232E71052320810745
:1001D000232291072324A1072326B1072328C1073F
:1001E000232AD107232CE107232EF107732520347E
:1001F000F3251034130601006F000000731015344E
:1002000083204100032181008321C10003220101D9
:1002100083224101032381018323C10103240102BD
:1002200083244102032581028325C10203260103A1
:1002300083264103032781038327C1030328010485
:1002400083284104032981048329C104032A010569
:10025000832A4105032B8105832BC105032C01064D
:10026000832C4106032D8106832DC106032E010731
:10027000832E4107032F8107832FC1071301C10775
:10028000730020302320C5006376B50013054500B8
:100290006FF05FFF678000000000000000000000BA
:1002A000000000000000000000000000000000004E
:1002B000130101F8232011002322210023243100FF
:1002C0002326410023285100232A6100232C71009A
:1002D000232E8100232091022322A1022324B10294
:1002E0002326C1022328D102232AE102232CF10272
:1002F000232E010323201105232221052324310568
:100300002326410523285105232A6105232C710545
:10031000232E8105232091072322A1072324B1073F
:100320002326C1072328D107232AE107232CF1071D
:100330009702020083A2421723A02200F322103466
:10034000232E5106EF00C03B170102000321C11507
:10035000032101008322C10773901234B7220000E9
:100360009382028873A00230832001000322C1001F
:100370008322010103234101832381010324C1015D
:100380008324010203254102832581020326C10241
:100390008326010303274103832781030328C10325
:1003A000832801040329410483298104032AC10409
:1003B000832A0105032B4105832B8105032CC105ED
:1003C000832C0106032D4106832D8106032EC106D1
:1003D000832E0107032F4107832F81071301010893
:1003E00073002030970202009382C21123A01200F2
:1003F00023A2220023A4320023A6420023A85200F5
:1004000023AA620023AC720023AE820023A09202D2
:1004100023A2A20223A4B20223A6C20223A8D202CC
:1004200023AAE20223ACF20223AE020323A01205A8
:1004300023A2220523A4320523A6420523A85205A0
:1004400023AA620523AC720523AE820523A092077E
:1004500023A2A20723A4B20723A6C20723A8D20778
:1004600023AAE20723ACF207EF7040321701020023
:1004700003218103032101008322C10773901234F9
:10048000B72200009382028873A00230832001000B
:100490000322C1008322010103234101832381013F
:1004A0000324C10183240102032541028325810223
:1004B0000326C10283260103032741038327810307
:1004C0000328C103832801040329410483298104EB
:1004D000032AC104832A0105032B4105832B8105CF
:1004E000032CC105832C0106032D4106832D8106B3
:1004F000032EC106832E0107032F4107832F810797
:10050000130101087300203097020200938282FFDA
:1005100083A0020003A1420083A1820003A2C200C3
:1005200083A2020103A3420183A3820103A4C201A7
:1005300083A4020203A5420283A5820203A6C2028B
:1005400083A6020303A7420383A7820303A8C2036F
:1005500083A8020403A9420483A9820403AAC20453
:1005600083AA020503AB420583AB820503ACC20537
:1005700083AC020603AD420683AD820603AEC2061B
:1005800083AE020703AFC20983AF82076780000012
:1005900073700430130101F823201100232221007D
:1005A000232431002326410023285100232A6100FF
:1005B000232C7100232E8100232091022322A102EB
:1005C0002324B1022326C1022328D102232AE102D7
:1005D000232CF102232E01032320110523222105C0
:1005E000232431052326410523285105232A6105AB
:1005F000232C7105232E8105232091072322A10797
:100600002324B1072326C1072328D107232AE10782
:10061000232CF1079702020083A202E923A0220003
:10062000232E1106EF30D033170102000321C1E75A
:10063000032101008322C10773901234B722000006
:100640009382028873A00230832001000322C1003C
:100650008322010103234101832381010324C1017A
:100660008324010203254102832581020326C1025E
:100670008326010303274103832781030328C10342
:10068000832801040329410483298104032AC10426
:10069000832A0105032B4105832B8105032CC1050A
:1006A000832C0106032D4106832D8106032EC106EE
:1006B000832E0107032F4107832F810713010108B0
:1006C00073002030737004306F00000073104530E9
:1006D000678000007325403073F04330678000006E
:1006E00097070000938747FE232EB5FE2322C5FA05
:1006F000232635F82320F5F8130505F86780000058
:10070000130101FF23261100EF700005EF20105C9C
:10071000631805008320C1001301010167800000F8
:100720008320C100130101016F309023130101FEEA
:10073000232631019309050013058003232A910024
:1007400023244101232E1100232C81002328210181
:100750002322510193840500130A0600EF50903BB9
:100760006304051297070200938707D083A7070049
:10077000130405006388070A639C040813094400F6
:100780001305090023269402231A04022328440394
:1007900023203401EF00005213058401EF00805143
:1007A00097070200938707CC03A707000325C4021D
:1007B00093072000B38497402328840023228402D7
:1007C000232C9400636AA70493172500B387A7001E
:1007D0009397270017050200130585DA3305F50006
:1007E00093050900EF00804D130510008320C1011F
:1007F0000324810183244101032901018329C100CC
:10080000032A8100832A410013010102678000004E
:10081000930410006FF09FF69707020023A4A7C46B
:100820006FF09FFA17050200130585D597070200A0
:1008300023AC87C2EF00004617050200130585D5DB
:10084000EF004045970A0200938A0AD613850A00F2
:10085000EF00404417090200130949D613050900A7
:10086000EF00404317050200130585D6EF008042D4
:100870009707020023AE57BF9707020023A827BFA0
:10088000E38E04EE6FF0DFF81305F0FF6FF01FF654
:10089000130101FE232A910023282101970402005D
:1008A000938484BC17090200130989BB83A7040041
:1008B000232C81000324090023263101232E11005B
:1008C000330485001385470093890500EF004047F6
:1008D00083A504008327090023A285006372F40422
:1008E00097070200938787B803A507009385450003
:1008F000EF00C03F6382090483A504000324810143
:100900008320C101832441010329010113850900CA
:100910008329C10093858501130101026F00003D09
:10092000970702009387C7B403A507009385450086
:10093000EF00C03BE39209FC8320C1010324810145
:1009400083244101032901018329C100130101020C
:1009500067800000130101FD23202103232E3101B4
:10096000232611022324810223229102232C4101F8
:10097000232A51012328610123267101170902004E
:10098000130909C08327090597090200938989ADD6
:1009900063800706737004308327C90503A4C7006A
:1009A00013058401EF00C0397360043093044400E0
:1009B00013850400EF00C0388327C40283A6090012
:1009C00093850400139527003305F50013152500C2
:1009D000130705003305A90063F2F61C1707020090
:1009E0002322F7A8EF00802D83270905E39407FA57
:1009F000EF20502197070200938747A603A707001F
:100A0000970A0200938ACAA583A70A003305E54026
:100A1000170702002322A7A4170A0200130A4AA5F7
:100A2000970B0200938B8BA4170B0200130BCBA226
:100A3000630A050C938717001305F5FF17070200DB
:100A40002320F7A2170702002328A7A003270A00E4
:100A5000639E070083A60B00170602002328E6A06A
:100A6000170702002326D7A0138706008326070056
:100A7000E38006FC0327C7000324C70003274400C4
:100A800063FEE7006FF0DFFA03A7C70083A70A0041
:100A90000324C7000327440063E2E70673700430B1
:100AA0009304440013850400EF0080298327840207
:100AB0001305840163840700EF008028736004300D
:100AC0008327C40203A70900938504001395270018
:100AD0003305F500131525003305A9006376F700EB
:100AE000170702002320F798EF00401D83270A0014
:100AF00003A70700E31A07F883A70A0003250B00E2
:100B0000E31A05F283A60900170702002328F794C9
:100B1000939726003387D700131727003307E90080
:100B200003270700631E0708638406049387F6FF04
:100B3000139727003307F700131727003307E9003F
:100B40000327070063160706638007029387E6FF03
:100B5000139727003307F700131727003307E9001F
:100B6000032707006316070417070200232CF78EDC
:100B70008320C1020324810283244102032901024C
:100B80008329C101032A8101832A4101032B010129
:100B9000832BC10013010103678000003305E900C6
:100BA000EF00C01183270905E39607DE6FF05FE4CD
:100BB00093860700170702002326F78A93972700DA
:100BC000B387D700939727003307F90083264700A0
:100BD000938787003309F90083A746002322F70093
:100BE0006382270503A5C700032481028320C10275
:100BF0009707020023AAA786832441020329010242
:100C00008329C101032A8101832A4101032B0101A8
:100C1000832BC10003230500832505031301010372
:100C20006700030083A747002322F7006FF09FFBB4
:100C3000130101FF232611002322910023248100A8
:100C40008327C50003A4C70093048401138504000F
:100C5000EF00000F93850400170502001305459768
:100C6000EF00C005970702009387078083A707005E
:100C70000325C4028320C10083A7C7020324810087
:100C8000832441003335F50013451500130101019C
:100C900067800000930785001307F0FF2322F5000B
:100CA0002324E5002326F5002328F5002320050052
:100CB0006780000023280500678000008327450027
:100CC00023A2F50003A7870023A4E50003A787005C
:100CD0002322B70023A4B70023A8A500832705007B
:100CE000938717002320F5006780000003A6050006
:100CF0009307F0FF130785006316F6006F0080036B
:100D0000138707008327470083A60700E37AD6FEF0
:100D100023A2F50023A4B70023A4E5002322B700F3
:100D200023A8A50083270500938717002320F5003B
:100D30006780000003270501832747006FF05FFDF0
:100D40000327450083268500832705012324D70038
:100D500003278500832645002322D70003A74700E9
:100D60006316A7000327850023A2E70023280500B8
:100D700003A507001305F5FF23A0A7006780000067
:100D80000326050493870500630406028325C50036
:100D900003274500B385C5002326B50063E6E500BB
:100DA000832505002326B500138507006F500077C3
:100DB00067800000130101FF232481002326110016
:100DC0001304050023229100EF30D06C83278404A4
:100DD000635AF004832744026386070493044402A1
:100DE0006F000002832784049387F7FF2324F40411
:100DF000832784046358F002832744026384070234
:100E000013850400EF301018E30E05FCEF30D044DA
:100E1000832784049387F7FF2324F404832784041F
:100E2000E34CF0FC9307F0FF2324F404EF30D06987
:100E3000EF30506683274404635AF004832704018B
:100E400063860704930404016F00000283274404AF
:100E50009387F7FF2322F404832744046358F002A6
:100E6000832704016384070213850400EF30901187
:100E7000E30E05FCEF30503E832744049387F7FFD1
:100E80002322F40483274404E34CF0FC9307F0FF8F
:100E90002322F404032481008320C1008324410021
:100EA000130101016F30506263000508130101FF57
:100EB000232481002322910013040500232611001E
:100EC00093840500EF30105D832604048327C40358
:100ED00003270400232C0402B387F6021306F0FF55
:100EE0002322C4042324E4002324C404B386D7406B
:100EF000B307F7003307D7002322F4002326E400CA
:100F00006398040283270401639E0702EF30D05BDD
:100F10008320C100032481008324410013051000B5
:100F20001301010167800000737004306F0000003E
:100F300013050401EFF01FD613054402EFF09FD50F
:100F40006FF0DFFC13050401EF30D00393071000AE
:100F5000E31EF5FAEFF0CFE36FF05FFB63160500D9
:100F6000737004306F000000130101FE232A91000A
:100F70002328210123263101232E1100232C810057
:100F8000930906001389050093040500638E050884
:100F90003305B50213055505EF50C037130405009E
:100FA000630C0508930745052320F500232E9402C2
:100FB00023202405EF30104E832604048327C40326
:100FC000032704001306F0FFB387F602232C040264
:100FD0002322C4042324E4002324C40413050401AD
:100FE000B386D740B307F7003307D7002322F400B6
:100FF0002326E400EFF01FCA13054402EFF09FC957
:10100000EF30904C23083405130504008320C10100
:101010000324810183244101032901018329C100A3
:10102000130101026780000013054005EF50802E78
:101030001304050063160500737004306F00000090
:10104000232084006FF09FF6631605007370043050
:101050006F0000006376B500737004306F0000000D
:10106000130101FF232481001306200013840500CF
:101070009305000023261100EFF05FEE630C0500DE
:10108000232C85028320C100032481001301010168
:1010900067800000737004306F000000130101FBD3
:1010A00023261104232481042322910423202105D3
:1010B000232E3103232C4103232A510323286103C8
:1010C000232671032326C10063060528638C0526A9
:1010D00093072000639CF6000327C50393071000C5
:1010E0006306F700737004306F0000001389060078
:1010F0009384050013040500EF30101A631A0500ED
:101100008327C10063860700737004306F000000FE
:10111000EF305038032784038327C403130B0000E8
:10112000930B20009309F0FF130A0401930A440271
:101130006364F710630479238327C1006382073651
:1011400063160B0013058101EF30807EEF30D0373E
:10115000EF20C029EF301034832744046394370113
:101160002322040483278404639437012324040482
:10117000EF3090359305C10013058101EF30407EBB
:1011800063160530EF301031032784038327C4032F
:101190006304F710EF305033EF30D02F83278404EF
:1011A0006346F0026F00000313850A00EF30805D94
:1011B00063040500EF30500A832784049387F7FF08
:1011C0002324F404832784046356F0008327440215
:1011D000E39C07FC23243405EF30102FEF30902BD5
:1011E000832744046346F0026F00000313050A00DE
:1011F000EF30405963040500EF30100683274404A4
:101200009387F7FF2322F404832744046356F000F6
:1012100083270401E39C07FC23223405EF30D02A06
:10122000EF204050130B1000EF30D026032784032B
:101230008327C403E370F7F0032604046304061253
:10124000631A091E0325840093850400EF50002DC6
:10125000832784008326040403274400B387D70030
:101260002324F40063E4E710832784038326040027
:1012700003274402938717002324D400232CF4026D
:101280006300071013054402EF30C04F93071000AE
:101290006318F50E6F004014EF3010238325C10052
:1012A00013050A00EF300021EF30D01E832784049D
:1012B0006346F0026F00000313850A00EF30804C94
:1012C00063040500EF304079832784049387F7FF98
:1012D0002324F404832784046356F0008327440204
:1012E000E39C07FC23243405EF30101EEF30901AE6
:1012F000832744046346F0026F00000313050A00CD
:10130000EF30404863040500EF3000758327440444
:101310009387F7FF2322F404832744046356F000E5
:1013200083270401E39C07FC23223405EF30D01906
:10133000EF20403FE31805EEEFF08FA5130B1000F0
:101340006FF09FEE83270504E38407D873700430A1
:101350006F000000737004306F0000000326040467
:101360006310060883270400638607048327840329
:101370000327440293871700232CF402E31407F099
:10138000EF309014130510008320C104032481045E
:1013900083244104032901048329C103032A81030F
:1013A000832A4103032B0103832BC102130101058F
:1013B0006780000003254400EF30D00083278403BA
:1013C000032744022322040093871700232CF402EE
:1013D000E31A07EAE30605FAEFF08F9B6FF05FFA76
:1013E0000325C40093850400EF50401383270404B1
:1013F0000327C40083260400B307F0403307F70037
:101400002326E400637ED70403274400B307F700D4
:101410002326F40013072000832744026304E90411
:101420000327840313071700232CE402E38A07F43D
:101430006FF05FE50325C40093850400EF50000EB4
:10144000832704040327C40083260400B307F04065
:101450003307F7002326E400E37ED7FA6FF0DFFAC4
:101460008327440203278403E30C07FA032784033A
:101470001307F7FF232CE402032784031307170045
:10148000232CE402E38E07EE6FF0DFDF1305040088
:10149000EFF05F92EF200029130500006FF0DFEE00
:1014A000EF309002130500006FF01FEE130101FFF3
:1014B0002322910093040500130540052324810095
:1014C00023261100EF40106513040500630C05048A
:1014D000232C05029307F0FF2322F50413071000C5
:1014E00013050501232EE4022324F404232204001F
:1014F00023200400232404002326040023200404C2
:1015000023089404EFF00FF913054402EFF08FF86D
:101510009306000013060000930500001305040065
:10152000EFF0DFB7130504008320C100032481001E
:101530008324410013010101678000006304050456
:10154000130101FF2324810023229100232611008F
:10155000232021010329450013040500EF30C05268
:10156000930400006304A9028320C10003248100C6
:1015700013850400032901008324410013010101A4
:1015800067800000737004306F0000008327C40080
:10159000930410009387F7FF2326F400E39607FCDB
:1015A00093060000130600009305000013050400D5
:1015B000EFF0DFAE6FF05FFB6302050A638805089A
:1015C000130101FE232C8100232A910023282101ED
:1015D00023244101232E11002326310193072000EB
:1015E0009384060013090600138A050013040500FE
:1015F000639CF6000327C503930710006302F70AF4
:10160000737004306F000000EFF0CF8C0327840369
:101610008327C403930905006366F704930400005D
:1016200013850900EFF08F8A8320C1010324810113
:101630001385040003290101832441018329C1008A
:10164000032A81001301010267800000832705043B
:10165000E38807F6737004306F0000007370043085
:101660006F00000003260404631E060C8327040099
:1016700063860712832784031307F0FF93871700FD
:10168000232CF402832784046388E70E83278404D1
:1016900093041000938717002324F4046FF05FF87D
:1016A000EFF04F83032784038327C40393090500C6
:1016B0006360F70603260404E30A06FA0325C40060
:1016C00093050A00EF409065832704040327C400B4
:1016D00083260400B307F0403307F7002326E40015
:1016E0006378D70003274400B307F7002326F400EC
:1016F00093072000E390F4F883278403E38C07F634
:10170000832784039387F7FF232CF4026FF09FF65F
:1017100003260404E30C06F40325C40093050A0021
:10172000EF40D05F832704040327C400832604000E
:10173000B307F0403307F7002326E400E364D7FA49
:101740006FF09FFBE39C04F60325840093050A00D9
:10175000EF40D05C832784008326040403274400E1
:10176000B387D7002324F400E3E6E7F083270400DF
:101770002324F4006FF01FF0832744029304100029
:10178000E38007EA13054402EF20D07FE30A05E86F
:10179000E30809E8232099006FF09FE8032544003F
:1017A000EF304042232204006FF0DFEC6302050AB1
:1017B0008327050463860700737004306F00000000
:1017C00083270500638A0708130101FE232C81008B
:1017D000232A910013040500232821012326310127
:1017E000232E110013890500EFE0DFEE03278403A9
:1017F0008327C40393090500930400006376F7026E
:10180000832784031307F0FF93871700232CF40228
:1018100083278404638AE7048327840493041000E5
:10182000938717002324F40413850900EFE01FEACF
:101830008320C101032481011385040003290101D0
:10184000832441018329C100130101026780000044
:10185000737004306F00000083274500E38607F6AD
:10186000737004306F000000832744026396070002
:10187000930410006FF05FFB13054402EF2090709B
:10188000E30805FEE30609FE930710002320F90094
:101890006FF01FFE130101FC232E1102232C810285
:1018A000232A9102232821032326310323244103E1
:1018B000232251032326C10063060528638C0526D5
:1018C000938A06009389050013040500EF30C01CBD
:1018D000631A05008327C100638607007370043014
:1018E0006F000000EF30003B832784036394071CE4
:1018F0008327C1006380071013058101EF30400387
:101900009304F0FF13094402130A0401EF30C03BB3
:10191000EF10D02DEF3000388327440463949700F4
:10192000232204048327840463949700232404045B
:10193000EF3080399305C10013058101EF3040027B
:1019400063100524EF30003583278403638A070A78
:10195000EF308037EF300034832784046346F00291
:101960006F00000313050900EF20D0616304050038
:10197000EF30800E832784049387F7FF2324F40439
:10198000832784046356F00083274402E39C07FC0A
:1019900023249404EF304033EF30C02F83274404D6
:1019A0006346F0026F00000313050A00EF20905D0C
:1019B00063040500EF30400A832744049387F7FF50
:1019C0002322F404832744046356F0008327040190
:1019D000E39C07FC23229404EF30002FEF10905477
:1019E000EF30402B832784036396070C8327C100C5
:1019F000E39E07F0EF30402D130500006F00800FCD
:101A0000EF30802C83270400638807108325C100F2
:101A100013050900EF20102AEF30C0278327840424
:101A20006346F0026F00000313050900EF20905594
:101A300063040500EF304002832784049387F7FF97
:101A40002324F404832784046356F000832744028C
:101A5000E39C07FC23249404EF300027EF3080231D
:101A6000832744046346F0026F00000313050A0055
:101A7000EF20505163040500EF20107E83274404BB
:101A80009387F7FF2322F404832744046356F0006E
:101A900083270401E39C07FC23229404EF30C02237
:101AA000EF10504863040508EF30C01E83278403FD
:101AB000E38E07F293850900130504008324C40014
:101AC000EFF00FAC63940A08832784030327040014
:101AD0009387F7FF232CF40263160700EF300026EC
:101AE0002322A4008327040163920708EF30C01D5E
:101AF000130510008320C1030324810383244103C1
:101B0000032901038329C102032A8102832A410296
:101B10001301010467800000EF30C0170325440063
:101B2000EF20507AEF30401A6FF05FEEEFE05FA6E3
:101B30006FF09FF783270504E38407D873700430A0
:101B40006F000000737004306F00000083274402B0
:101B500023269400E38C07F813054402EF209042FB
:101B6000E30605F8EFE0DFA26FF05FF8130504016C
:101B7000EF20504193071000E31AF5F66FF09FFE37
:101B800013050400EFF00FA3EF10D0391305000088
:101B90006FF05FF663000506130101FF2324810047
:101BA00023202101232611002322910083244500B4
:101BB0001389050013040500EF20106D6380A40451
:101BC00093060000130609009305000013050400A6
:101BD000EFF05FCC93071000630CF5028320C10087
:101BE0000324810083244100032901001301010122
:101BF00067800000737004306F0000008327C4000A
:101C000013051000938717002326F4006FF01FFDC3
:101C10008327C400938717002326F4006FF01FFC6E
:101C2000630805066386050C130101FE232C810061
:101C3000232A910023282101232631012324410155
:101C400013040500232E11001309060093890500D3
:101C5000EFE05FA883278403130A050093040000C4
:101C6000639C070213050A00EFE05FA68320C10111
:101C70000324810113850400032901018324410108
:101C80008329C100032A810013010102678000003B
:101C9000737004306F00000003260404630406021E
:101CA0008325C40083274400B385C5002326B400E0
:101CB00063E6F500832504002326B400138509009C
:101CC000EF40D005832784031307F0FF9387F7FFC6
:101CD000232CF402832744046384E702832744040B
:101CE00093041000938717002322F4046FF09FF7EA
:101CF00083270504E38A07F2737004306F00000045
:101D00008327040163960700930410006FF09FF58A
:101D100013050401EF201027E30805FEE30609FE82
:101D2000930710002320F9006FF01FFE63060508DB
:101D300083270504638A050863840708130101FEED
:101D4000232C8100232A91002328210123244101EF
:101D500013040500232E110023263101138A0500E8
:101D6000EFE05F97832784031309050093040000C5
:101D7000638E07008329C40093050A00130504003D
:101D8000EFF00F809304100023263401130509009F
:101D9000EFE0DF938320C101032481011385040058
:101DA00003290101832441018329C100032A810001
:101DB0001301010267800000737004306F0000009F
:101DC000737004306F000000E38C07FE7370043002
:101DD0006F00000063160500737004306F00000090
:101DE000130101FF232481001304050023261100A1
:101DF000EF20506A03248403EF20106D8320C1007C
:101E00001305040003248100130101016780000011
:101E100063160500737004306F000000130101FFAA
:101E2000232611002324810013040500EF2090666F
:101E3000832784030324C4033304F440EF20D068D1
:101E4000130504008320C100032481001301010154
:101E50006780000063060500032585036780000096
:101E6000737004306F000000630805049787030057
:101E70009387479403A747006304E50403A7C700BB
:101E80006302E50803A74701630AE50603A7C70144
:101E90006302E50603A74702630AE50403A7C70236
:101EA0006302E50403A74703630AE50203A7C70328
:101EB0006302E5026F40005E737004306F00000043
:101EC0001307000013173700B387E70023A00700AC
:101ED0006F40405C130770006FF0DFFE1307600077
:101EE0006FF05FFE130750006FF0DFFD1307400037
:101EF0006FF05FFD130730006FF0DFFC1307200069
:101F00006FF05FFC130710006FF0DFFB0325C504C3
:101F1000678000002326B50467800000034505059F
:101F2000678000006308050003258503133515004D
:101F300067800000737004306F000000630C0500C0
:101F4000832785030325C5033305F54013351500A5
:101F500067800000737004306F000000130101FF00
:101F60002324810023229100232021012326110014
:101F700013040500138905009304060073700430F0
:101F8000EF205051032784038327C4036306F70817
:101F9000EF20905373600430737004300327840380
:101FA0008327C403130500006360F70273600430E5
:101FB0008320C10003248100832441000329010000
:101FC000130101016780000003260404630A06066A
:101FD0000325840093050900EF40405483278400C3
:101FE0008326040403274400B387D7002324F40086
:101FF00063E6E700832704002324F4008327840397
:102000000327440293871700232CF4026316070466
:10201000130510006FF09FF9EF20104B6398040434
:10202000736004308320C1000324810083244100B5
:10203000032901001305000013010101678000005E
:1020400083270400E39C07FA03254400EF20903720
:10205000232204006FF09FFA13054402EFE05FBDF6
:10206000E30805FA1305B0FF6FF05FF49305040170
:1020700013850400EFE0DF81736004301305C0FFB7
:102080006FF01FF3130101FF2324810023261100A9
:1020900013040500737004308327850363900702DF
:1020A0006310060A736004308320C100032481009A
:1020B0001305000013010101678000007360043004
:1020C000737004308327850313050000639C0700A9
:1020D000736004308320C1000324810013010101D7
:1020E0006780000013870500032604048325C400CD
:1020F00083274400B385C5002326B40063E6F500BA
:10210000832504002326B4008327840313050700D6
:102110009387F7FF232CF402EF404040832704010C
:1021200063960700130510006FF09FFA1305040172
:10213000EFE01FB0E30805FE1305B0FF6FF05FF995
:102140009305450213050600EFE08FF47360043039
:102150001305C0FF6FF01FF8130101FF2322910048
:102160002326110023248100032785038327C50329
:1021700093040600636EF7008320C10003248100EE
:1021800013850400832441001301010167800000CE
:102190000326050413040500630A060403258500CD
:1021A000EF40C037832784008326040403274400BC
:1021B000B387D7002324F40063E6E70083270400F5
:1021C0002324F4008327840393871700232CF4022D
:1021D000E39404FA83274402E38007FA13054402D8
:1021E000EFE01FA5B334A0006FF01FF983270500AF
:1021F000E39A07FC03254500EF20D01C23220400AE
:102200006FF05FFC8327850363820708130101FFDA
:102210002326110023248100232291008327C50057
:102220000328050403274500B38707012326F5008B
:1022300063E6E700832705002326F5008326850350
:1022400013870500938507009387F6FF232CF5027B
:102250009304060013040500130608001305070085
:10226000EF40C02B83A70400639607008327040177
:10227000639207028320C10003248100832441006C
:102280001305100013010101678000001305000011
:102290006780000013050401EFE09F99E30C05FC43
:1022A0009307100023A0F4006FF0DFFC9777030082
:1022B0009387475003A707006300070403A787001D
:1022C0006308070403A707016308070403A787013E
:1022D0006308070403A707026308070403A787022C
:1022E0006308070403A70703630C070403A7870316
:1022F000630407046780000013070000131737000A
:10230000B387E70023A0B70023A2A70067800000DF
:10231000130710006FF09FFE130720006FF01FFEE1
:10232000130730006FF09FFD130740006FF01FFD93
:10233000130750006FF09FFC130770006FF01FFC35
:10234000130760006FF09FFB977703009387874622
:1023500003A747006300E50403A7C7006306E5047D
:1023600003A747016306E50403A7C7016306E50465
:1023700003A747026306E50403A7C7026306E50453
:1023800003A74703630AE50403A7C7036302A7047F
:10239000678000001307000013173700B387E700BA
:1023A00023A0070067800000130710006FF0DFFE16
:1023B000130720006FF05FFE130730006FF0DFFDA2
:1023C000130740006FF05FFD130750006FF0DFFC54
:1023D000130770006FF05FFC130760006FF0DFFB06
:1023E000130101FF232481002322910023202101D6
:1023F0001304050023261100938405001309060029
:10240000EF205009032744049307F0FF6314F700FB
:1024100023220404032784049307F0FF6314F700C6
:1024200023240404EF20500A83278403639A0700BF
:10243000130609009385040013054402EF20C0230E
:10244000EF20500583278404635AF0048327440255
:1024500063860704930444026F0000028327840408
:102460009387F7FF2324F404832784046358F0023E
:10247000832744026384070213850400EF20803021
:10248000E30E05FCEF20405D832784049387F7FF6C
:102490002324F40483278404E34CF0FC9307F0FF27
:1024A0002324F404EF205002EF20C07E832744044D
:1024B000635AF0048327040163860704930404012C
:1024C0006F000002832744049387F7FF2322F4045C
:1024D000832744046358F0028327040163840702BE
:1024E00013850400EF20002AE30E05FCEF20C05600
:1024F000832744049387F7FF2322F40483274404AB
:10250000E34CF0FC9307F0FF2322F4040324810042
:102510008320C1008324410003290100130101012C
:102520006F20807A63040504130101FD232E31011D
:10253000232C410123261102138A07002324810240
:102540002322910223202103232A51012328610100
:10255000232671012324810193079000930907002A
:1025600063FAE700737004306F000000737004308A
:102570006F000000930A050093840500130906000C
:10258000938B0600130B08006304082C1305000648
:10259000EF305058130405006304052A131929006D
:1025A00023286503130609009305500A13050B0041
:1025B000EF40C00803C70400832704031309C9FFC1
:1025C000230AE40203C70400338927011379C9FFF2
:1025D0006306070E83C71400A30AF40283C714001E
:1025E000638E070C83C72400230BF40283C72400E7
:1025F0006386070C83C73400A30BF40283C734003F
:10260000638E070A83C74400230CF40283C7440087
:102610006386070A83C75400A30CF40283C75400DF
:10262000638E070883C76400230DF40283C7640028
:102630006386070883C77400A30DF40283C7740080
:10264000638E070683C78400230EF40283C78400C9
:102650006386070683C79400A30EF40283C7940021
:10266000638E070483C7A400230FF40283C7A4006A
:102670006386070483C7B400A30FF40283C7B400C2
:10268000638E070283C7C4002300F40483C7C40019
:102690006386070283C7D400A300F40483C7D40071
:1026A000638E070083C7E4002301F40483C7E400BA
:1026B0006386070083C7F400A301F404130B4400EE
:1026C00013050B00A3010404232634032328340537
:1026D000232A0404EFE00FDE13058401EFE08FDD11
:1026E0009307A000B3873741232C040423288400D8
:1026F000232CF4002322840223220404232E040426
:1027000013860B0093850A0013050900EFD05FFDC7
:102710002320A40063040A0023208A00737004307D
:1027200017E90100130989D68327090097E40100FE
:10273000938484D7638C070003A7040083A7040055
:1027400083274704938717002322F70417E7010024
:10275000130787D4832707009387170097E60100A4
:1027600023ACF6D283A704006380071083270900F7
:1027700017EA0100130A0AE7639C070083A7040015
:1027800083A7C70263E6F90097E7010023AE87D06D
:1027900097E70100938787CE03A7070097E601001C
:1027A000938606CF8327C40283A60600130717006B
:1027B00017E601002324E6CC2324E40463F6F600A4
:1027C00017E701002326F7CC13074001B387E70280
:1027D00093050B003305FA00EFE04FCE8327090085
:1027E0006388070083A7040083A74704639E070844
:1027F0008327090013041000638A070083A70400DD
:1028000083A7C70263F43701EFD09FD813050400F4
:102810008320C1020324810283244102032901028F
:102820008329C101032A8101832A4101032B01016C
:10283000832BC100032C810013010103678000007A
:1028400013050B00EF3010451304F0FF6FF01FFC71
:1028500013152600EF30102C130B0500E31805D2DA
:102860001304F0FF6FF09FFA97E7010023AE87C2D1
:102870000327070093071000630AF70217EA010015
:10288000130A4AD66FF0DFF003A7040083A6040002
:10289000832747049387F7FF2322F70483A746047F
:1028A000E39807F4736004306FF09FF4930A00001C
:1028B00017EA0100130A0AD3130C4001930BA0007E
:1028C00033858A03938A1A003305AA00EFE08FBC90
:1028D000E3987AFF97EB0100938B4BDD13850B0098
:1028E000EFE04FBB97EA0100938A8ADD13850A0067
:1028F000EFE04FBA17E501001305C5DDEFE08FB932
:1029000017E50100130545DEEFE0CFB817E501003C
:102910001305C5DEEFE00FB897E7010023A477B9F0
:1029200097E7010023AE57B76FF09FE6130101FF51
:10293000232481002326110023229100232021013A
:10294000130405007370043097E40100938404B409
:1029500083A70400639E07106318040097E7010033
:10296000938787B403A407001309440013050900E3
:10297000EFE00FBD832784026386070013058401FF
:10298000EFE00FBC9305090017E501001305C5D55D
:10299000EFE0CFB297E70100938747B003A70700A6
:1029A00097E70100938787AD83A7070013071700F8
:1029B00097E6010023A4E6AE03A70400938717005F
:1029C00097E6010023ACF6AA630C070097E7010025
:1029D000938787AD03A7070003274704631C070EEF
:1029E00083A70400638A070697E701009387C7ABB4
:1029F00003A70700630287107370043003A7040065
:102A00006318070817E701001307C7A98326070003
:102A100083A606006392060A1307F0FF97E60100FB
:102A200023ACE6A403A704006308070203A707007A
:102A3000032747046302070203A7070083A60700D2
:102A4000832747049387F7FF2322F70483A74604CD
:102A500063940700736004308320C1000324810065
:102A60008324410003290100130101016780000054
:102A700097E70100938747A303A7070083A70700F1
:102A800083274704938717002322F7046FF0DFECB6
:102A900083A6070003A7070003A746041307170030
:102AA00023A2E60417E701001307C79F8326070048
:102AB00083A60600E38206F6032707000327C70064
:102AC0000327C7000327470097E6010023A6E69ADD
:102AD0006FF05FF503A7070083A60700832747046D
:102AE0009387F7FF2322F70483A74604E39A07EEB0
:102AF000736004306FF0DFEE97E7010093878797EC
:102B000083A7070063860700737004306F0000001E
:102B1000032481008320C100832441000329010094
:102B2000130101016FD0DFA66304050C17E7010054
:102B30001307879783260700930700006386A60A7A
:102B4000130101FF23261100232481002322910079
:102B50007370043097E601009386469383A70600BE
:102B6000638C07000326070083270700832746049A
:102B7000938717002322F60483A706009304050019
:102B800003244501638807008327070083A74704C0
:102B90006394070697E701009387C79083A7070010
:102BA000638C870697E701009387878F83A70700C9
:102BB0006384870697E70100938747B46306F404AC
:102BC00097E70100938747B2630CF4029307100064
:102BD0008320C10003248100832441001385070062
:102BE0001301010167800000138507006780000062
:102BF000737004306F000000EF5090626FF09FF927
:102C0000930740006FF0DFFC83A7840293B717009F
:102C1000938727006FF0DFFB930720006FF05FFBC7
:102C20007370043097E701009387478603A7070076
:102C3000631607026304050483A707000325C50282
:102C4000638C070097E701009387078603A70700B7
:102C500003274704631C07026780000017E7010091
:102C600013078784832607000327070003A746046A
:102C70001307170023A2E604E31005FC17E7010081
:102C800013078782032507006FF01FFB03A70700C8
:102C900083A60700832747049387F7FF2322F704BF
:102CA00083A74604E39A07FA736004306780000044
:102CB000130101FF232481001304050023261100C2
:102CC000EFD05FA16318040097D701009387C77DF9
:102CD00003A407000324C402EFD05F9F8320C10038
:102CE0001305040003248100130101016780000023
:102CF0009307900063F6B700737004306F00000014
:102D0000130101FE232C8100232E1100232A9100A0
:102D10002328210123263101232441011304050026
:102D20007370043017D9010013094976832709000D
:102D3000639207106300041283270405638EF50A6B
:102D400017D701001307477663F0B7028326070001
:102D5000638E8612032707008324C702B3B495004D
:102D600093C414006F00000183240700B3848440DF
:102D700093B414000327C4026386E70E83278401FB
:102D80002328B40463C807009307A000B385B740A5
:102D9000232CB40093172700B387E70003274401CF
:102DA00097E901009389098493972700B387F90075
:102DB0006310F704130A440013050A00EFD05FF80C
:102DC00017D701001307C76C8327C4020327070026
:102DD0006376F70017D70100232CF76A1307400129
:102DE000B387E70293050A003385F900EFD01FEDA2
:102DF00063840400EFD0CFF983270900638C0700B8
:102E000097D701009387476A83A7070083A74704E2
:102E1000639E07048320C1010324810183244101AF
:102E2000032901018329C100032A81001301010242
:102E30006780000097D701009387076703A7070003
:102E400083A7070083274704938717002322F704EB
:102E5000E31404EE97D701009387076503A40700E6
:102E60006FF09FED2326B4026FF05FF10324810120
:102E70008320C10183244101032901018329C10069
:102E8000032A8100130101026F509039930400005E
:102E90006FF05FEE630A0508130101FE232A91001B
:102EA00097D401009384446083A70400232E11006B
:102EB000232C810023282101232631016388A704C4
:102EC0007370043017D901001309495C8327090086
:102ED000638C070003A7040083A70400832747042B
:102EE000938717002322F7040327450197E7010082
:102EF0009387C780630EF702832709006388070062
:102F000083A7040083A74704639E07088320C101A9
:102F10000324810183244101032901018329C10084
:102F20001301010267800000737004306F0000001D
:102F30008327850217D701001307C779E38EE7FAC5
:102F4000E39C07FA93094500130405001385090063
:102F5000EFD01FDF17D70100130787538327C40261
:102F6000032707006376F70017D701002322F752E3
:102F700013074001B387E70217D5010013058566E3
:102F8000938509003305F500EFD05FD383A70400D4
:102F90000327C40283A7C702E360F7F6EFD04FDF31
:102FA0006FF09FF5032481018320C1018324410137
:102FB000032901018329C100130101026F5050262A
:102FC00063020506130101FE232C8100232A9100D0
:102FD0002328210113040500232E1100232631018B
:102FE000EFD04FEF0327440197D701009387077174
:102FF0001309050093040000630AF7021305090092
:10300000EFD0CFEC8320C10103248101138504009C
:1030100003290101832441018329C1001301010215
:1030200067800000737004306F0000008327840203
:1030300017D501001305056AE382A7FCE39007FC9E
:1030400097D701009387074383A707006394070678
:1030500097D701009387474583A707008324C402BD
:103060009309440083A7C70213850900B3B4F40091
:10307000EFD01FCD17D70100130787418327C40264
:103080000327070093C414006376F70017D70100E5
:103090002320F74013074001B387E70217D501004B
:1030A00013054554938509003305F500EFD01FC182
:1030B0006FF0DFF493058401EFD05FC06FF01FF471
:1030C000130101FE37150000232E1100232C81006F
:1030D000232A9100232821012326310123244101A1
:1030E0002322510123206101EF30C0226308052211
:1030F0009304050013050006EF30C02113040500FA
:1031000063040526371600009305500A232895020C
:1031100013850400EF30805283240403B7170000A6
:103120009387C7FFB384F400B7474C459387974410
:10313000130A4400232AF40213050A00230C040294
:10314000A30104042326040223280404232A0404DC
:10315000EFD05FB613058401EFD0DFB59307A00071
:10316000232C040493F4C4FF23288400232CF400AC
:103170002322840223220404232E040413060000C5
:10318000971500009385C5EA13850400EFD04FD54D
:103190002320A4007370043017D901001309092FEC
:1031A0008327090097D4010093840430638C0700BF
:1031B00003A7040083A7040083274704938717000D
:1031C0002322F70417D701001307072D83270700D1
:1031D0009387170097D6010023A0F62C83A704003D
:1031E0006388070A8327090097D901009389893FDB
:1031F000639C070083A7040083A7C70263960700A8
:1032000097D7010023A2872A97D701009387072722
:1032100003A7070097D60100938686278327C40259
:1032200083A606001307170017D601002328E624FB
:103230002324E40463F6F60017D70100232AF724B9
:10324000139527003305F5001315250093050A0093
:103250003385A900EFD09FA6832709006388070064
:1032600083A7040083A74704639E070C83270900F4
:103270006384070083A70400EF2050069307100023
:10328000630AF510631C0508737004306F000000BA
:1032900097D7010023AA8720032707009307100070
:1032A00097D9010093890934E310F7F6938A09004E
:1032B00017DB0100130B8B3F13850A00938A4A0129
:1032C000EFD05F9DE31A5BFF17D501001305053EA4
:1032D000EFD05F9C97DA0100938A8A3E13850A003B
:1032E000EFD05F9B17D501001305C53EEFD09F9A25
:1032F00017D501001305453FEFD0DF9917D5010021
:103300001305C53FEFD01F9997D7010023AC67196C
:1033100097D7010023A657196FF01FEF8320C10133
:103320000324810183244101032901018329C10070
:10333000032A8100832A4100032B010013010102AB
:103340006780000003A7040083A6040083274704C6
:103350009387F7FF2322F70483A74604E39807F037
:10336000736004306FF09FF0032481018320C1015A
:10337000032901018329C100032A8100832A410016
:10338000032B010013850400832441011301010272
:103390006F304010737004309307F0FF17D70100AF
:1033A000232CF70C0324810197D7010023A0A70E3B
:1033B0008320C10183244101032901018329C10024
:1033C000032A8100832A4100032B010097D70100C3
:1033D00023A2070C130101026FD0CF807370043059
:1033E00097D7010023A4070A6FD00F9217D70100C7
:1033F0001307470883270700938717002320F70048
:10340000678000007370043097D701009387070826
:1034100003A707006318070217D7010013078707E0
:103420000325070083A70700638C070097D70100D7
:103430009387870703A7070003274704631407023E
:103440006780000017D701001307070683260700CF
:103450000327070003A746041307170023A2E60467
:103460006FF09FFB03A7070083A60700832747048D
:103470009387F7FF2322F70483A74604E39207FC10
:103480007360043067800000130101FF23261100E0
:1034900023248100EFD00FA497D70100938787FFE3
:1034A00003A40700EFD08FA28320C10013050400FE
:1034B00003248100130101016780000097D70100F8
:1034C000938787FD03A5070067800000130101FDB6
:1034D0002326110223248102232291022320210387
:1034E000232E3101232C4101232A5101232861017C
:1034F0002326710197D701009387C7F783A7070099
:10350000639A070617D701001307C7F88327070038
:103510009387170097D6010023AEF6F6832A07009B
:10352000638A0A0A97D70100938707F583A70700E4
:103530009304000063FEFA0A97D901009389890A6F
:1035400017DA0100130A4AF683270A0093061000CF
:1035500003A7C70293172700B387E70093972700B5
:10356000B389F90083A7090063F4F60293041000FD
:103570006F00000297D70100938707F183A7070028
:10358000930400009387170017D70100232EF7EE4E
:1035900097D70100938707EF83A70700638407008D
:1035A000930410008320C1020324810213850400C8
:1035B00003290102832441028329C101032A8101D5
:1035C000832A4101032B0101832BC1001301010355
:1035D0006780000017D401001304C4EC83270400A3
:1035E00083A707006388070C737004306F00000026
:1035F00017D40100130404EB97D90100938989FEC5
:1036000017DA0100130A4AEA17DB0100130B4BE833
:103610008327040083A7070063800708832704002B
:1036200083A7C70003A9C70083274900930B49005C
:1036300013850B0063EAFA06EFD08FF08327890227
:103640001305890163840700EFD08FEF8327C90238
:1036500003270B0093850B00139527003305F50016
:10366000131525003385A9006376F70017D70100ED
:103670002320F7E2EFD08FE483270A000327C90253
:1036800083A7C702E366F7F88327040093041000BA
:1036900083A70700E39407F89307F0FF17D701000B
:1036A000232CF7DC6FF05FEA17D701002326F7DC45
:1036B0006FF09FE917D70100130787DE8327040007
:1036C0000327070097D6010023AEE6DC17D70100D9
:1036D0002328F7DC97D70100938787DA83A70700B1
:1036E0009387170017D70100232CF7D883270400EE
:1036F00083A70700639A07009307F0FF17D701001D
:10370000232CF7D66FF01FE28327040083A7C7009E
:1037100083A7C70083A7470017D70100232EF7D43C
:103720006FF05FE097D701009387C7D403A7070026
:1037300063160700737004306F000000130101FE70
:10374000232E1100232C8100232A910023282101FC
:103750002326310123244101232251012320610129
:103760007370043097D40100938444D203A70400FB
:103770006310071203A707001307F7FF97D601008E
:1037800023AAE6CE83A70700639E070A97D7010006
:10379000938787D083A707006386070A97DA01001B
:1037A000938A4AE417DA0100130A8ACE17D9010076
:1037B000130989CF930910006F00C0013385EA0017
:1037C000EFD0CFCF832709000327C40283A7C70206
:1037D0006374F70683A70A0F6380070E83A7CA0FD7
:1037E00003A4C70013058401EFD08FD5130B440049
:1037F00013050B00EFD0CFD48327C40283260A0021
:1038000093050B00139527003305F50013152500CC
:10381000130705003385AA00E3F2F6FA17D7010073
:103820002328F7C6EFD08FC9832709000327C402D6
:1038300083A7C702E360F7FA97D7010023A437C52F
:103840006FF05FF91304000083A70400638C070086
:1038500097D70100938747C583A7070083A747042D
:1038600063980704130504008320C1010324810128
:1038700083244101032901018329C100032A810016
:10388000832A4100032B010013010102678000001D
:1038900017D70100130747C1832607000327070036
:1038A00003A746041307170023A2E6046FF09FEC5A
:1038B000EF5000176FF01FFB17D401001304C4BCB6
:1038C00083270400638C0702832704001309100078
:1038D00063860702EFF09FBF6306050097D70100DC
:1038E00023A227BB832704009387F7FF17D7010084
:1038F000232CF7B883270400E39E07FC97D7010029
:10390000938747B803A7070093071000E31CF7F25B
:10391000EFC01FC8130410006FF01FF3630405020B
:1039200063960500737004306F00000017D7010024
:10393000130747B483270700638A070073700430B6
:103940006F000000737004306F000000130101FF6E
:103950002324810023261100832607000327050066
:103960009386160017D601002326D6B097D60100FD
:10397000938646B283A606003304B7002320850051
:1039800063F0E6046372E40263F0860297D70100F5
:10399000938787B103A5070013054500EFD04FBA01
:1039A00013050400EF40507FEFF0DFD7630E0500F2
:1039B0008320C100032481001301010167800000FE
:1039C000E366E4FC6FF05FFC032481008320C10008
:1039D000130101016FC0DFBB630E050017D70100A3
:1039E000130747A983270700638807007370043013
:1039F0006F0000006FC0DFB9130101FF2326110023
:103A000023248100032707009307050013071700ED
:103A100097D6010023A0E6A697D601009386C6A8F4
:103A200017D70100130707A70327070003A5060000
:103A30003304F70013054500EFD08FB013050400E1
:103A4000EF409075EFF01FCE631A0500032481004C
:103A50008320C100130101016FC09FB38320C10007
:103A6000032481001301010167800000130101FF9D
:103A7000232481002326110097D701009387879F75
:103A800083A70700130400009387170017D70100CE
:103A90002322F79E97D70100938707A083A70700EB
:103AA00063EEF51417DE0100130E8EBF97D20100EE
:103AB000938282B21304000013070000930F1000DA
:103AC0001303500A6F00C000130ECEFE6384C20FB2
:103AD00083278EFF93060700E38807FE8327CEFF28
:103AE00083A74700232EFEFE6386C71303AFC700DC
:103AF00083A747003307E500930E0000232EFEFE48
:103B00006380C70983A8C700938748032320170150
:103B10002322F70083A788042326F7012324F70034
:103B200083A7C8022328F70083A70805232C0700D2
:103B3000232AF70003A80803834708006398670453
:103B4000930708009387170083C60700B3850741D2
:103B5000E38A66FE93D525009395050193D505016B
:103B6000231EB700938E1E0013070702630A1F036C
:103B70008327CEFF83A74700232EFEFEE394C7F9D9
:103B800083274E00232EFEFE6FF0DFF79305000023
:103B9000231EB700938E1E0013070702E31A1FFDB2
:103BA0003304D40113175400130ECEFE93060700FE
:103BB000E390C2F397D701009387C78E03AE070047
:103BC00083270E006396071297D701009387478DCE
:103BD00003AE070083270E00639A071C17DE01005F
:103BE000130E4EA083274E10639C070283278E116D
:103BF000639C07266304060023200600EFF09FB2B3
:103C0000130504008320C100032481001301010176
:103C10006780000083274E00232EFEFE6FF01FED0D
:103C200083278E1017DF0100130F8FAC83A7470087
:103C300017D70100232CF7AA6386E73D83A2C700AC
:103C400083A74700B306D500930E000017D70100E5
:103C5000232EF7A8930F40001303500A6382E7094D
:103C600083A8C7009387480323A0160123A2F60068
:103C700083A7880423A6F60123A4F60083A7C8021D
:103C800023A8F60083A7080523AC060023AAF600A4
:103C900003A8080383470800639A67329307080064
:103CA0009387170003C70700B3850741E30A67FE40
:103CB00093D725009397070193D70701239EF6001A
:103CC000938E1E0093860602638C123183278E101A
:103CD00083A7470017D70100232AF7A0E392E7F94B
:103CE00083270E1117D701002322F7A06FF05FF78B
:103CF00083274E00130F8E0083A647002322DE0089
:103D00006380E633B307E50003A7460083A2C6003D
:103D1000930E00002322EE00930F20001303500A9D
:103D20006300EF088328C7001387480323A0170107
:103D300023A2E70003A7880423A6F70123A4E70032
:103D400003A7C80223A8E70003A7080523AC0700C0
:103D500023AAE70003A8080303470800631E67229D
:103D6000130708001307170083460700B305074130
:103D7000E38A66FE13D725001317070113570701BF
:103D8000239EE700938E1E00938707026380122311
:103D900083264E0003A746002322EE00E314EFF82B
:103DA0000327CE002322EE006FF0DFF783274E00BB
:103DB000130F8E0083A747002322FE00638CE725A4
:103DC00083A2C70083A74700B306D500930E000067
:103DD0002322FE00930F20001303500A6300FF0804
:103DE00083A8C7009387480323A0160123A2F600E7
:103DF00083A7880423A6F60123A4F60083A7C8029C
:103E000023A8F60083A7080523AC060023AAF60022
:103E100003A8080383470800639867149307080002
:103E20009387170003C70700B3850741E30A67FEBE
:103E300093D725009397070193D70701239EF60098
:103E4000938E1E0093860602638A121383274E0008
:103E500083A747002322FE00E314FFF88327CE0048
:103E60002322FE006FF0DFF78327CE1197DE0100DB
:103E7000938E4E8983A7470017D701002322F78826
:103E8000638AD71783AFC70083A747003307D500DE
:103E90001303000097D6010023A4F686130F300009
:103EA000930220009308500A6388D70903A5C7002E
:103EB000930745032320A7002322F70083278504C7
:103EC0002326E7012324F7008327C5022328F700D0
:103ED000832785026384070023265700832705056F
:103EE000232C0700232AF700032805038347080033
:103EF000639C1705930708009387170083C6070084
:103F0000B3850741E38A16FF93D7250093970701EE
:103F100093D70701231EF7001303130013070702AB
:103F2000638EAF028327CE1183A7470097C6010097
:103F300023A8F67CE39CD7F783274E1297C601008F
:103F400023A0F67C6FF09FF693070000231EF70076
:103F50001303130013070702E396AFFC3304640056
:103F6000E31C06C86FF09FC993070000239EF6006C
:103F7000938E1E0093860602E39A12ED17CE01007F
:103F8000130E4E6683274E103304D401931654004B
:103F9000E38E07C46FF0DFC813070000239EE7001D
:103FA000938E1E0093870702E39412DF97C70100E8
:103FB0009387074F03AE07003304D40193165400D0
:103FC00083270E00E38C07C06FF05FDE93070000CD
:103FD000239EF600938E1E0093860602E39812CF6E
:103FE00083278E113304D40193165400E38407C051
:103FF0006FF09FE783274E1217C701002322F77047
:104000006FF05FE883270E1117C701002320F76EBA
:104010006FF0DFC28327CE002322FE006FF05FDA4D
:104020008326CE002322DE006FF0DFCD130101FDD9
:104030002322910223202103232E3101232C41012D
:10404000232A51012328610123267101232611020D
:104050002324810297C901009389C94117C901002E
:104060001309495817CA0100130A4A4297CA0100A6
:10407000938A8A4397CB0100938B0B4297C401002C
:104080009384C441130B10006F00000283A7090042
:10409000032449109387170017C70100232CF73C0E
:1040A000EFF04FE8631E040083A70400E39007FECF
:1040B00083270900E37AFBFEEFC08FCD6FF0DFFEB0
:1040C0007370043083270A00639E07048327091155
:1040D00003A4C70013054400EFC09FC683A70B00CD
:1040E0009387F7FF17C701002328F73A83A7040037
:1040F0009387F7FF17C701002322F73A83270A00A7
:104100006388070083A70A0083A747046398070210
:1041100003250403EF20003813050400EF20803747
:104120006FF09FF803A70A0083A70A0083274704BC
:10413000938717002322F7046FF05FF903A70A00A3
:1041400083A60A00832747049387F7FF2322F704F7
:1041500083A74604E39E07FA736004306FF05FFBA9
:1041600097C701009387073183A707006396070E5F
:10417000130101FF2326110097C7010023A4073074
:1041800017C701001307473283270700B7A6A5A565
:104190009386565A83A7070383A50700639ED5001D
:1041A00003A64700631AB60083A687006396C6007D
:1041B00083A7C700638AD70003250700832507006C
:1041C00093854503EF30407697C601009386462CD1
:1041D00003A6060017C701001307C7406F000002BF
:1041E00083A706006382070883A706009387F7FF6B
:1041F00017C60100232EF62803A6060093172600F3
:10420000B387C70093972700B307F70083A707007A
:10421000E38807FC03A6060093172600B387C700B0
:1042200093972700B305F70083A64500938787007F
:10423000B307F70083A6460023A2D500638AF602DF
:1042400083A7C6008320C10017C70100232EF724CF
:1042500013010101678000009307100017C70100D8
:104260002322F72267800000737004306F00000083
:10427000930740013306F60283A646003307C700C2
:104280002322D7006FF0DFFB130101FE2328210159
:10429000232E1100232C8100232A91002326310193
:1042A000130905007370043097C401009384041E41
:1042B00083A7040017C401001304041F639C070CA8
:1042C00063140900032904009309490013850900B8
:1042D000EFC01FA7832789026386070013058901A2
:1042E000EFC01FA69385090017C5010013050541FE
:1042F000EFC0DF9C83A704006388070083270400C6
:1043000083A747046394070A832704006384270D67
:1043100083A70400638207067370043083A7040038
:104320006398070E97C701009387C71703A7070075
:10433000032707006310070C9307F0FF17C701005E
:10434000232CF71283A70400638807028327040045
:1043500083A747046382070203270400832604001F
:10436000832747049387F7FF2322F70483A7460494
:1043700063940700736004308320C101032481012A
:1043800083244101032901018329C1001301010292
:104390006780000003270400832704008327470465
:1043A000938717002322F7046FF09FF1032704007F
:1043B00083260400832747049387F7FF2322F7040B
:1043C00083A74604E39207F4736004308327040054
:1043D000E39027F583A704006382070697C70100CF
:1043E0009387470983A707006388070A737004301F
:1043F0006F00000083A7070083A7C70083A7C7003B
:1044000083A7470017C701002328F7066FF09FF323
:10441000032704008327040083274704938717009A
:104420002322F70497C701009387C70703A7070054
:1044300003270700E30207F06FF0DFFB97C70100D7
:104440009387870517C701001307C71983A70700BC
:10445000032787116314F7028320C101032481011C
:1044600097C7010023A20704832441010329010106
:104470008329C10013010102678000000324810128
:104480008320C10183244101032901018329C10043
:10449000130101026FF0DFCC032481018320C101ED
:1044A00083244101032901018329C1001301010271
:1044B0006FC00F8E6306050A130101FF23229100CE
:1044C00097C40100938444FE232021011389050031
:1044D00083A50400232611002324810093858501F0
:1044E000EFC0DF8003A5040013054500EFC05F8522
:1044F0009307F0FF630AF90697C70100938787F9CE
:1045000003A4070003A7040083A7070033042401C2
:1045100023228700636EF40697C70100938787F80C
:1045200003A5070083A5040093854500EFC00FFC99
:1045300097C70100938747F483A707006376F400C9
:1045400097C7010023AA87F28320C10003248100BA
:104550008324410003290100130101016780000049
:10456000737004306F00000083A5040003248100F1
:104570008320C100832441000329010017C50100E5
:104580001305C51793854500130101016FC00FF393
:1045900097C701009387C7F003A507000324810094
:1045A00083A504008320C100832441000329010066
:1045B00093854500130101016FC04FF3630E0500A1
:1045C00097C70100938707EB83A70700639A07004B
:1045D000737004306F000000737004306F000000CF
:1045E000130101FF2322910097C401009384C4EBBF
:1045F00003A704009387050083A50400B706008085
:10460000B3E7D7002326110023248100232CF700D1
:104610009385850113040600EFC04FEA03A504004B
:1046200013054500EFC0CFF19307F0FF6304F402D8
:1046300097C70100938707E603A507008320C10001
:104640008324410033058500032481001301010107
:104650006F40803483A50400032481008320C100BF
:104660008324410017C501001305450993854500C2
:10467000130101016FC08FE46308050A130101FFF4
:104680002322910097C40100938404E22320210196
:104690001389050083A5040023261100232481002B
:1046A0009385850113040600EFC04FE103A50400C4
:1046B00013054500EFC0CFE893071000630AF40626
:1046C00097C70100938707DD03A4070003A7040031
:1046D00083A707003304240123228700636EF406B6
:1046E00097C70100938707DC03A5070083A5040093
:1046F00093854500EFC08FDF97C701009387C7D729
:1047000083A707006376F40097C7010023A687D626
:104710008320C10003248100832441000329010078
:104720001301010167800000737004306F00000006
:1047300083A50400032481008320C1008324410059
:104740000329010017C50100130545FB93854500AA
:10475000130101016FC08FD697C70100938747D41B
:1047600003A507000324810083A504008320C10062
:1047700083244100032901009385450013010101B1
:104780006FC0CFD6130101FF23261100232481001F
:10479000232291008327C50003A4C7006304040AF1
:1047A0009304840113850400EFC08FD997C70100DB
:1047B000938747CC83A70700639A070893044400B4
:1047C00013850400EFC0CFD797C70100938747CC6C
:1047D0000327C40283A7070063F6E70097C7010019
:1047E00023A8E7CA93172700B387E700939727000A
:1047F00017C50100130505DF938504003305F50097
:10480000EFC0CFCB97C70100938707CA83A70700E4
:104810000327C4021305000083A7C70263FAE70059
:104820009307100017C70100232EF7C413051000CB
:104830008320C1000324810083244100130101016E
:1048400067800000737004306F00000093850400DF
:1048500017C50100130505E8EFC04FC66FF09FFABA
:1048600097C70100938707C183A7070063960700D6
:10487000737004306F000000130101FF2326110044
:104880002324810023229100B70700800324C50060
:10489000B3E7F5002320F50063080408EFC04FCA12
:1048A0009304440013850400EFC08FC997C701002B
:1048B000938707BE0327C40283A7070063F6E700B8
:1048C00097C7010023A6E7BC93172700B387E7002B
:1048D0009397270017C501001305C5D03305F500D0
:1048E00093850400EFC08FBD97C701009387C7BBB6
:1048F00083A707000327C4021305000083A7C7028C
:1049000063FAE7009307100017C70100232CF7B6DE
:10491000130510008320C10003248100832441007B
:104920001301010167800000737004306F00000004
:104930006304050297C70100938787B403A70700A4
:1049400097C70100938707B583A707002320E500D9
:104950002322F50067800000737004306F000000B0
:104960006304050E638E050C130101FF232611005D
:1049700023248100130705007370043097C80100D9
:104980009388C8B083A708006380070297C7010017
:10499000938787B183A6070083A7070083A74604F0
:1049A0009387170023A2F60417C30100130383AEF5
:1049B00083A70500032603009306F0FF13040000FD
:1049C0006388D70417CE0100130E8EAB03250E00AB
:1049D00003280700832647006306A800130410007D
:1049E0006378D6023308D640130410006372F802CD
:1049F00003250E00B387C74003260300B387D70003
:104A000023A0F5002320A7002322C70013040000E1
:104A100083A70800638C070097C701009387C7A886
:104A200083A7070083A747046394070213050400C4
:104A30008320C1000324810013010101678000006D
:104A4000737004306F000000737004306F0000005A
:104A5000EF30107D6FF09FFD9307100017C7010026
:104A60002322F7A267800000630605000325C50422
:104A700067800000130500006780000063040500E4
:104A80002326B5046780000097C701009387C7A15C
:104A900003A507006780000097C701009387079F61
:104AA00083A7070013051000638C070097C7010058
:104AB0009387479C03A507001335150013151500B0
:104AC00067800000630C0508130101FE232A910092
:104AD00097C401009384449D83A70400232E1100F2
:104AE000232C810023282101232631010327C5021D
:104AF00083A7C7026376F7048327850163CC070089
:104B000083A7040083A6C7029307A000B387D740FA
:104B1000232CF50093172700B387E70003274501EF
:104B200017C90100130909AC93972700B307F900CF
:104B30006308F70283A7040083A7C7022326F502B0
:104B40008320C10103248101832441010329010140
:104B50008329C10013010102678000006780000003
:104B6000930945001304050013850900EFC04F9D0C
:104B700083A7040017C701001307879103270700C5
:104B800083A7C7022326F4026376F70017C7010044
:104B90002320F790139527003305F50003248101A6
:104BA000131525008320C101832441019385090049
:104BB0003305A9008329C100032901011301010262
:104BC0006FC0CF8F63060502130101FF232611007A
:104BD000232481002322910097C701009387C78C6B
:104BE00003A40700630AA400737004306F00000080
:104BF00013050000678000008327440563960700C3
:104C0000737004306F0000008326C402032704057C
:104C10009387F7FF232AF4046384E600638E07007A
:104C2000130500008320C100032481008324410078
:104C30001301010167800000930444001385040000
:104C4000EFC00F908327040517C70100130747849F
:104C5000832607001307A0003307F7402326F4023A
:104C6000232CE40063F6F60017C701002322F78225
:104C700013074001B387E70217C5010013058596A6
:104C8000938504003305F500EFC04F831305100032
:104C90006FF05FF97370043097B701009387077F57
:104CA00083A707006380070297B701009387C77F38
:104CB00003A7070083A707008327470493871700EC
:104CC0002322F7046780000097B701009387077CD1
:104CD00083A70700638C070297B701009387C77CFF
:104CE00003A70700032747046302070203A707007F
:104CF00083A60700832747049387F7FF2322F7043F
:104D000083A7460463940700736004306780000043
:104D100097B701009387477903A6070083A607008A
:104D200003A707009307A00083A6C60203258601F8
:104D3000B387D740232CF7006780000097B70100A6
:104D40009387877603A70700630A070083A60700F7
:104D500003A746051307170023AAE60403A50700C7
:104D600067800000130101FD232021032326110287
:104D70002324810223229102232E310113090500ED
:104D80007370043097B401009384447083A70400C7
:104D900017B4010013044471639E070A83270400BB
:104DA00083A78705639A0700832704001307100071
:104DB00023AEE704639A050E83A704006388070007
:104DC0008327040083A74704639A07147370043091
:104DD00083A70400639407068327040003A58705BF
:104DE00063080500630209048327040023AC070459
:104DF0008327040023AE070483A704006388070009
:104E00008327040083A74704639207068320C10217
:104E10000324810283244102032901028329C10161
:104E2000130101036780000003270400832787051F
:104E30009387F7FF232CF7046FF09FFB03270400F1
:104E40008327040083274704938717002322F7044E
:104E50006FF09FF80327040083270400832747048B
:104E6000938717002322F7046FF05FF303270400F2
:104E700083260400832747049387F7FF2322F70440
:104E800083A74604E39407F8736004308320C102CB
:104E90000324810283244102032901028329C101E1
:104EA0001301010367800000032504002326B100DD
:104EB00013054500EFB0DFE88325C1009307F0FF3D
:104EC0006380F50897B701009387C75C83A9070043
:104ED0000327040083A70700B389B9002322370101
:104EE00063ECF90697B701009387C75B03A507003A
:104EF0008325040093854500EFB05FDF97B701007D
:104F00009387875783A7070063F6F90097B70100D7
:104F100023A43757EFB0CFE76FF01FEA0327040051
:104F200083260400832747049387F7FF2322F7048F
:104F300083A74604E39C07E8736004306FF01FE921
:104F40008325040017B501001305457B93854500B3
:104F5000EFB0DFD66FF01FFC97B70100938747547F
:104F600003A507008325040093854500EFB01FD8F3
:104F70006FF05FFA130101FD23202103232E31017D
:104F8000232611022324810223229102232C410192
:104F900013890500930906007370043097B401006B
:104FA0009384C44E83A7040017B401001304C44FB4
:104FB000639C071403270400930720000327C705F9
:104FC0006304F702832704001345F5FF03A7870551
:104FD0003375E50023ACA7048327040013071000F2
:104FE00023AEE704639A060A83A7040063880700D8
:104FF0008327040083A74704639407167370043063
:1050000083A70400639E07066388090083270400C2
:1050100083A7870523A0F900032704009307100046
:10502000130500000327C705630EF700832704005C
:105030001349F9FF1305100003A787053379E90029
:1050400023AC27058327040023AE070483A70400AD
:10505000638807008327040083A747046392070C33
:105060008320C10203248102832441020329010217
:105070008329C101032A8101130101036780000014
:10508000032704008327040083274704938717001E
:105090002322F7046FF05FF7032504002326D100D5
:1050A00013054500EFB0DFC98326C1009307F0FF69
:1050B000638AF60C97B701009387C73D03AA0700E0
:1050C0000327040083A70700330ADA0023224701DD
:1050D0006368FA0C97B701009387C73C03A50700E4
:1050E0008325040093854500EFB05FC097B70100AA
:1050F0009387873883A707006370FA0A97B7010080
:1051000023AC47376F0040090327040083270400BE
:1051100083274704938717002322F7046FF09FE942
:105120000327040083260400832747049387F7FF9F
:105130002322F70483A74604E39407F27360043044
:105140008320C10203248102832441020329010236
:105150008329C101032A8101130101036780000033
:105160000327040083260400832747049387F7FF5F
:105170002322F70483A74604E39207E87360043010
:105180006FF0DFE78325040017B50100130505570D
:1051900093854500EFB09FB2EFB08FBF6FF0DFE4B3
:1051A00097B701009387C72F03A507008325040045
:1051B00093854500EFB09FB36FF01FFE630A050CA7
:1051C000130101FF232611002324810023229100D3
:1051D000232021017370043097B401009384042BC1
:1051E00083A7040063960708638606008327850566
:1051F00023A0F60093070600930620000326C505AA
:10520000232ED50413870500130405006382D70AF3
:1052100063F4F608930530006388B70093054000F7
:105220006396B700630CD610232CE4049307100098
:10523000630CF6081304100083A70400638C0700B6
:1052400097B701009387472683A7070083A74704E2
:1052500063980706130504008320C100032481001E
:10526000832441000329010013010101678000002C
:1052700097B701009387472303A7070083A7070079
:1052800083274704938717002322F7046FF0DFF585
:10529000737004306F00000093061000E398D7F895
:1052A0008327850533E7B700232CE5046FF01FF84B
:1052B0008327850593871700232CF5046FF01FF7CC
:1052C000EF3000766FF01FF9130944001305090051
:1052D000EFB01FA717B701001307871B8327C4026E
:1052E000032707006376F70017B701002322F71A98
:1052F00013074001B387E70217B501001305852E98
:10530000930509003305F500EFB05F9B8327840206
:1053100063860700737004306F00000097B70100C8
:105320009387871883A707000327C40283A7C702B0
:10533000E3F2E7F0EFB0CFA56FF0DFEF130400006A
:105340006FF09FEF63080508130101FE232C810015
:10535000232A9100232821012326310123244101FE
:1053600023225101232E110093090700138A0600FE
:10537000930406001389050013040500EFB08FB5F0
:10538000930A050063060A00832784052320FA0098
:105390000327C40593072000232EF4046380F4043C
:1053A00063FA9710930630006388D4009306400098
:1053B0006396D400630CF70E232C2405930710008A
:1053C0006312F70A83278402638207027370043032
:1053D0006F000000737004306F00000083278405A5
:1053E00093871700232CF4046FF05FFD97B701003B
:1053F0009387470883A707006390070A9304440034
:1054000013850400EFB0DF9317B7010013074708B7
:105410008327C402032707006376F70017B701004C
:105420002328F70613074001B387E70217B50100E9
:105430001305451B938504003305F500EFB01F8865
:1054400097B701009387470683A707000327C40285
:1054500083A7C70263F8E70063860900930710007B
:1054600023A0F9001304100013850A00EFB00FA663
:10547000130504008320C101032481018324410119
:10548000032901018329C100032A8100832A4100E5
:1054900013010102678000009305840117B5010024
:1054A00013054523EFB09F816FF09FF913040000AF
:1054B0006FF09FFB93071000E392F4F083278405BD
:1054C00033E92701232C24056FF05FEF630A050EF3
:1054D000130101FE232C8100232A910013040500EF
:1054E00023282101232E1100232631019384050056
:1054F000EFB04F9E930720008326C405232EF404AB
:1055000083278405130710001309050093871700EC
:10551000232CF4046396E60883278402638607003D
:10552000737004306F00000097B70100938787F411
:1055300083A70700639A07089309440013850900AD
:10554000EFB01F8017B70100130787F48327C40249
:10555000032707006376F70017B70100232AF7F245
:1055600013074001B387E70217B50100130585074C
:10557000938509003305F500EFB04FF497B70100AC
:10558000938787F283A707000327C40283A7C70274
:1055900063F8E700638604009307100023A0F4007B
:1055A000032481018320C101832441018329C10097
:1055B0001305090003290101130101026FB00F91C6
:1055C000737004306F0000009305840117B501006B
:1055D00013054510EFB08FEE6FF05FFA93070500EB
:1055E000630805067370043017B70100130707EA54
:1055F00083260700639E060203A6C70593062000C4
:10560000130500006316D60023AE0704130510002F
:1056100083270700638C070097B701009387C7E8CB
:1056200003A7070003274704631C070267800000E5
:1056300097B60100938646E703A6060083A60600F8
:1056400083264604938616002322D6046FF0DFFAE1
:1056500097B70100938747E583A707006FF09FF88E
:1056600003A7070083A60700832747049387F7FF54
:105670002322F70483A74604E39A07FA73600430F1
:1056800067800000130101FB2322910423202105E0
:10569000232C4103232A510323286103232671036A
:1056A0002326110423248104232E31032324810380
:1056B000232291032320A10317B901001309C9DF95
:1056C00017BB0100130B8BDE97B40100938444DEFB
:1056D00097BA0100938A0ADE130A1000930B900018
:1056E0008327090003A707006306071683A7C700DF
:1056F00083A90700EFD09FCFEFD0DFD083270B0027
:10570000130C05006368F50C97B7010023A0A7DA16
:10571000130600006376352303A50400B385894191
:10572000EFC01FCCEFE00F806306051603A5040051
:10573000930600001306000093058100EFC08F95CB
:10574000E30005FA83278100E3C207FE83290101F4
:1057500083A749016386070013854900EFB04FDE38
:10576000EFD05FCA83270B00130C05006362F50CB2
:105770008327810017B70100232A87D3E3E8FBFAC8
:10578000B317FA0013F707216310072013F7770CFC
:105790006316072A93F70702E38A07F813850900BF
:1057A000EF00504F6FF09FF883A7C70003A4C70016
:1057B00083AC07009309440013850900EFB04FD86C
:1057C0008327440213050400E78007008327C401F0
:1057D0006386470D8327090003A70700E31607FC2C
:1057E00003A70A0097B6010023A286CD97B6010051
:1057F00023A2F6CC97B7010023A0E7CCEFD09FF20D
:105800006FF0DFF283A7C70003A4C70003AD070052
:10581000930C440013850C00EFB08FD28327440211
:1058200013050400E78007008327C401638C470B3E
:105830008327090003A70700E31607FC03A70A0054
:1058400097B6010023A8F6C697B7010023A6E7C6BE
:105850006FF01FF2EFD09FB9EFD0DFBA83270B00B4
:10586000130C0500E368F5F683A70A0003A50400FE
:105870009309000003A60700B385894117B701000B
:10588000232687C313361600EFC09FB5EFD09FE9DC
:10589000E31E05E8EFA0DFCF6FF05FE98327840107
:1058A00093850900B387FC0063E2FC0883A704002A
:1058B00063860702232A0100232C9101232E8100F5
:1058C000EFF08F9D03A5040093060000130600006F
:1058D00093054101EFB08FFCE31E05EE73700430B9
:1058E0006F0000008327840193850C00B307FD003F
:1058F0006362FD0883A7040063860702232A010070
:10590000232CA101232E8100EFF00F9903A50400A1
:10591000930600001306000093054101EFB00FF855
:10592000E31805F0737004306F00000003250900D0
:105930002322F40023288400EFB04FBB6FF09FE9CF
:10594000EFD05FDE8327090083A7C70003A4C70049
:10595000930C440013850C00EFB08FBE8327C40165
:10596000638A47058327440213050400E780070084
:105970006FF0DFDB032509002322F40023288400D5
:10598000EFB0CFB66FF0DFEA8327C10023ACF90098
:105990006382070AB387870123A2F90023A839018C
:1059A000938549006362FC0803A50A00EFB00FB4B9
:1059B0006FF0DFD783278401232884003387F90021
:1059C0002322E400636AEC04330C3C41636EFC0266
:1059D00083A7040063860702232A0100232C3101D8
:1059E000232E8100EFF04F8B03A5040093060000E7
:1059F0001306000093054101EFB04FEAE31405F6EA
:105A0000737004306F00000003A50A0093850C003A
:105A1000EFB0CFAD6FF01FF50325090093850C00A3
:105A2000EFB0CFAC6FF01FF403250900EFB00FAC5F
:105A30006FF0DFCF737004306F0000008327C10068
:105A400083A6890123A839013387D70023A2E9005F
:105A50006362EC06B307FC4063EAD70683A74902FA
:105A600013850900E780070083A7C901E39047CDAC
:105A700083A689018327C10003A70400B387D70049
:105A800063060702232A0100232CF100232E310193
:105A9000EFF08F8003A504009306000013060000BA
:105AA00093054101EFB08FDFE31205C87370043036
:105AB0006F0000006374FC00E372F7FA032509002D
:105AC00093854900EFB08FA26FF05FC603A50A006F
:105AD00093854900EFB08FA16FF05FC5130101FFFF
:105AE0002324810023261100232291002320210159
:105AF00017B401001304C49BEFF0CF99832704006F
:105B000063840704EFF04F9C83270400638A070235
:105B100093080000130800009307000013072000FB
:105B2000930600001306004097B501009385058990
:105B300017050000130545B5EFC0DF9E6314050689
:105B4000737004306F00000017B90100130949BCDD
:105B500013050900EFB00F9497B40100938484BC3F
:105B600013850400EFB00F93130600009305C000E7
:105B70001305400097B7010023A0279597B70100B0
:105B800023AA9792EFB08FBD17B701002322A792E7
:105B90006306050297B501009385C581EFC00FF13B
:105BA0006FF05FF68320C10003248100832441004D
:105BB00003290100130101016780000073700430A4
:105BC0006F000000638A050A130101FD232A5101B9
:105BD000930A05001305C0022324810223229102A7
:105BE00023202103232E3101232C410123261102DE
:105BF00023286101232671011309070093890600F8
:105C0000130A060093840500EF00C070130405001A
:105C1000630C0502EFF00F8897B70100938747895F
:105C200083A70700638E0704EFF00F8A1305440073
:105C300023205401232C9400232E440123203403D9
:105C400023222403EFB00F87130504008320C10231
:105C50000324810283244102032901028329C10113
:105C6000032A8101832A4101032B0101832BC100F7
:105C70001301010367800000737004306F0000009F
:105C800097BB0100938BCBA813850B00EFB08F80DF
:105C900017BB0100130B0BA913050B00EFA09FFF0F
:105CA000130600009305C0001305400097B70100DC
:105CB00023A4778197A7010023AE677FEFB00FAAD7
:105CC00017A701002326A77E630A050097A50100F8
:105CD0009385456EEFC08FDD6FF01FF57370043054
:105CE0006F000000630E0506130101FE232C8100E6
:105CF000232E1100232A910017A401001304447BD2
:105D000083280400130805001305000063800804BD
:105D1000930407002322B100138706002324C10047
:105D2000232601019306500063C0B604EFE0DFD6DE
:105D300093072000630EF50403250400930600007A
:105D40001306000093054100EFB04FB58320C10159
:105D500003248101832441011301010267800000B3
:105D6000737004306F00000093054100930600003B
:105D70001306070013850800EFB01F848320C101BC
:105D80000324810183244101130101026780000083
:105D900003250400930600001386040093054100C8
:105DA000EFB0CFAF6FF09FFA630605000325050043
:105DB00067800000737004306F00000063160500F8
:105DC000737004306F000000130101FF23261100DF
:105DD0002324810013040500EFE0DFEB03254401D9
:105DE0003334A000EFE05FEE130504008320C10010
:105DF0000324810013010101678000006316050080
:105E0000737004306F000000130101FF2324810030
:105E10001304050023261100EFE0DFE7032404024A
:105E2000EFE09FEA8320C1001305040003248100F2
:105E300013010101678000006316050073700430D0
:105E40006F000000130101FF232481002322910031
:105E5000138405009304050023261100EFE09FE35F
:105E600023A08402032481008320C10083244100F5
:105E7000130101016FE05FE5130101FF1305C0018C
:105E80002324810023261100EF00C04813040500DD
:105E9000630805002320050013054500EFA09FDFE0
:105EA000130504008320C1000324810013010101B4
:105EB0006780000063020502B70700FFB3F7F50033
:105EC00063860700737004306F000000639A05005A
:105ED000737004306F000000737004306F000000B6
:105EE000130101FE232C81002328210123263101E7
:105EF0002324410123225101232E1100232A910042
:105F00009309070013890600930A0600138405000D
:105F1000130A0500EFE05FB8631805006386090007
:105F2000737004306F000000EFD04FCC83240A0060
:105F3000B3779400631209046382070463880A003C
:105F40009347F4FFB3F797002320FA00EFD08FFDBB
:105F50008320C10103248101138504000329010169
:105F6000832441018329C100032A8100832A41003F
:105F70001301010267800000E302F4FCE38809FCDE
:105F8000B33550019395850163060900B7070004F6
:105F9000B3E5F50013860900B3E5850013054A0053
:105FA000EFE0CFE1EFD00FF863140500EFA04FDE74
:105FB000EFE01FD6931765009309050063DA070029
:105FC000B70400019384F4FFB3F499006FF05FF815
:105FD000EFE05FCC83290A00B37734016310090234
:105FE000638A070063880A009347F4FFB3F7370119
:105FF0002320FA00EFE05FCD6FF09FFCE31CF4FE7E
:106000006FF05FFE630C0500B70700FFB3F7F50004
:10601000638A0700737004306F00000073700430EF
:106020006F000000130101FF232481001304050009
:10603000232611002322910023202101138905002A
:10604000EFE05FC5832404009345F9FFB3F79500A3
:106050002320F400EFE05FC78320C1000324810008
:106060001385040003290100832441001301010169
:1060700067800000130101FF232481001304050041
:1060800023261100EFA00FE503240400EFA00FE486
:106090008320C100130504000324810013010101C2
:1060A00067800000630C0500370700FFB3F7E500C9
:1060B000638A0700737004306F000000737004304F
:1060C0006F0000006F209018B70700FFB377F6004D
:1060D00063860700737004306F00000063160600CB
:1060E000737004306F000000130101FE232C810047
:1060F000232821012326310123244101232E1100CD
:10610000232A91001389060093890500130A0500CC
:1061100013040600EFE05F98631E050463060900A0
:10612000737004306F000000EFD04FAC83240A007E
:106130009385090013050A00B3E49900EFF09FF678
:10614000B3779400630AF40883240A00EFD08FDD4C
:106150008320C10103248101138504000329010167
:10616000832441018329C100032A81001301010214
:1061700067800000EFD08FA783240A009385090071
:1061800013050A00B3E43401EFF0DFF1B3F7840044
:1061900063848704E30A09FAB705000513060900BA
:1061A000B365B40013054A00EFE04FC1EFD08FD7BD
:1061B00063140500EFA0CFBDEFE09FB59317650016
:1061C0009304050063D40702B70700019387F7FF24
:1061D000B3F4F4006FF0DFF783270A001344F4FFF1
:1061E000B3F787002320FA006FF05FF6EFE09FAA75
:1061F00083240A00B3779400639887009347F4FFE1
:10620000B3F797002320FA00EFE01FAC6FF0DFFB3D
:10621000130101FF2324810023261100130405002C
:1062200023229100EFD08F9C8327440063860702CE
:10623000032504019304C400631895006F008003D4
:106240000325040163089502B7050002EFE04FE162
:1062500083274400E39607FE13050400EF00802324
:10626000032481008320C100832441001301010124
:106270006FD04FCB737004306F000000630C0500CB
:10628000370700FFB3F7E500638A07007370043037
:106290006F000000737004306F0000006F20007BFF
:1062A000630C0500B70700FFB3F7F500638A07002A
:1062B000737004306F000000737004306F000000D2
:1062C000130101FF232481002322910023261100C2
:1062D0001304050093840500EFE0DF9B032704000F
:1062E00093C7F4FFB377F7002320F4000324810061
:1062F0008320C10083244100130101016FE0DF9C72
:106300006306050003258501678000001305000072
:1063100067800000130101FF232481002326110060
:1063200013040500EFD08F8C97A7010093870719FE
:1063300083A70700639C0704B797010017A7010014
:106340001307C73F9387C7FF97A6010023AEE61642
:1063500017A701002328F71617A701002322F73EED
:1063600097A701009387C71517A701002328F73CBB
:106370009307100017A70100232A071417A701008D
:106380002320071417A70100232AF712631204021F
:10639000EFD04FB9EF10805813040000130504002C
:1063A0008320C100032481001301010167800000E4
:1063B00013058400937735006398070CB7970100A5
:1063C0001307F5FF9387A7FFE3E4E7FC97A6010017
:1063D0009386860F83A706006F00400103A707007E
:1063E000630A0700938607009307070003A7470087
:1063F000E366A7FE17A701001307870CE38AE7F8F7
:1064000003A70700130600011384870023A0E600FA
:1064100003A74700B306A740637ED6023388A700D0
:106420002322D80023A2A7008325480097A60100B5
:10643000938686096F0080009306070003A7060075
:1064400003264700E36AB6FE2320E80023A00601E6
:1064500003A7470097A701009387070983A70700B1
:10646000B387E74017A701002320F708EFD08FABD1
:10647000E30204F2130504008320C1000324810019
:1064800013010101678000001375C5FF1305450066
:106490006FF0DFF263080506130101FF232481007A
:1064A0002326110013040500EFC05FF4930584FF59
:1064B0000326C4FF17A70100130707016F00800020
:1064C000138707008327070083A64700E3EAC6FE79
:1064D000232CF4FE2320B70097A701009387C70061
:1064E00003A707008327C4FF032481008320C10082
:1064F000B387E70017A701002328F7FE1301010166
:106500006FD04FA26780000097A701009387C7FD57
:1065100003A5070067800000678000003367B500AF
:106520001377370093070500631207049308D6FF1B
:10653000B30815011307050093860500637815035A
:1065400003A806001307470093864600232E07FF83
:10655000E36817FF9347F5FFB387170193F7C7FF6A
:1065600093874700B385F500B307F5003306C500F0
:1065700063F4C70C9386450013884700B3B6D70071
:1065800033B8050133E7F50093C616001348180029
:1065900013773700B3E60601133717003377D700B8
:1065A000330EF64093861700630807061337AE00D4
:1065B0006314070613532E00138805009386070003
:1065C000130700008328080013071700130848006A
:1065D00023A0160193864600E36667FE1377CEFF7D
:1065E000B385E500B387E7006306EE0483C60500C4
:1065F000138717002380D700637EC70283C6150068
:1066000013872700A380D7006376C70203C725003E
:106610002381E70067800000B307F640B387F500E9
:106620009385150003C7F5FF93861600238FE6FEBA
:10663000E398F5FE6780000067800000B367C5003F
:1066400093F73700B308C5006382070E6376151110
:10665000B307A04093F73700138737009306500025
:1066600093F5F50F130815003383A8401306F6FFC2
:106670006374D700130750006368E60E6380070E4B
:106680002300B50013071000638EE700A300B500D8
:1066900013073000130825006396E7001308350040
:1066A0002301B5001396850033E6C5001397050155
:1066B0003367E6003303F34093968501B366D70052
:1066C00013562300B307F5001307000023A0D700DB
:1066D0001307170093874700E36AC7FE1377C3FFCA
:1066E000B307E8006300E3082380B70013871700AF
:1066F000637C1703A380B700138727006376170313
:106700002381B7001387370063701703A381B70095
:1067100013874700637A17012382B7001387570056
:1067200063741701A382B7006780000093F5F50F2B
:1067300013978500B365B700139705013367B7005A
:10674000E37415FF930705009387470023AEE7FE28
:10675000E3EC17FF67800000678000001308050066
:106760006FF05FF467800000930705006FF0DFF7BC
:106770008347050013070500638C07001305150008
:1067800083470500E39C07FE3305E5406780000072
:106790001305000067800000130515008347F5FF0F
:1067A0009385150003C7F5FF63880700E386E7FEBE
:1067B0003385E74067800000930700006FF05FFFBC
:1067C000930705009385150003C7F5FF938717000E
:1067D000A38FE7FEE31807FE6780000083460500ED
:1067E000930700026398F600130515008346050021
:1067F000E38CF6FE938756FD93F7D70F638007046B
:106800009307050093050000638806041305000044
:1068100093871700138606FD1317250083C607000C
:106820003305A700131515003305A600E39206FEF5
:10683000638405003305A04067800000938536FD22
:106840008346150093B5150093071500E39006FCE9
:10685000130500006FF0DFFD1305000067800000E6
:1068600083A705002380A70083A70500938717004F
:1068700023A0F5006780000097A60100938646C517
:1068800083A70600173703001307C7EB138617000B
:10689000B307F7002380A70097A5010023AAC5C26C
:1068A0009307A000630AF500930700046308F6004D
:1068B0001305000067800000E30C06FE370610F0A9
:1068C000130717008347F7FF2320F6F083A706007E
:1068D0009387F7FF97A5010023ACF5BEE39207FE6F
:1068E0001305000067800000130101EB23229114BF
:1068F00023202115232A5113232481132326111425
:1069000023248114232E3113232C411323286113B4
:1069100023267113232291132320A113232EB111B7
:1069200093040500138905002326C100130C5002AF
:10693000930A90008347090063888703638C0706E6
:1069400003A404006F008000638607062300F400A0
:1069500003A40400130919001304140023A08400E5
:1069600083470900E39287FF034619009308190043
:1069700093860800130D00029309F0FF130AF0FF3D
:1069800013080000130550059307D6FD93F7F70F82
:1069900013891600636EF53A17970100130787668F
:1069A00093972700B387E70083A70700B387E70023
:1069B000678007008320C1140324811483244114B9
:1069C000032901148329C113032A8113832A411344
:1069D000032B0113832BC112032C8112832C411230
:1069E000032D0112832DC1111301011567800000D1
:1069F000930C8000232401009307100063DA071D25
:106A00008327C10003A40400938B770093F68BFFC8
:106A100003AB060083A94600938786002326F10076
:106A200013860C009306000013050B0093850900E4
:106A3000EF1090352328A1009307000063803733BF
:106A4000930D4101930B100013860C009306000078
:106A500013050B0093850900EF10C06F930600002B
:106A600013860C00130B050093890500EF10D0313D
:106A70008327810023A0AD0093861B00938D4D00DA
:106A800063863701938B06006FF01FFCE37C9BFF4E
:106A900063D24603930704002380A70103A40400E4
:106AA000130AFAFF9307140023A0F40013840700CD
:106AB000E3C446FF93962B0093070101B386D700EA
:106AC0006F008002938777052300F40003A404007D
:106AD000938BFBFF93871B001304140023A08400F7
:106AE0009386C6FFE358F0E483A70600E3ECFAFCC4
:106AF000938707036FF05FFD83A7040093060003ED
:106B00000327C1002380D70083A704009306470012
:106B1000930C00011386170023A0C40013068007FE
:106B2000A380C70003A404002324010093070700E7
:106B30001304140023A0840003AB07009309000092
:106B40002326D1006FF0DFED8327C10083AC07005F
:106B5000938B470063880C28635C40259307D00221
:106B6000631EFD2083C70C006388070263D80924D5
:106B700083A60400938C1C00130AFAFF2380F600FE
:106B800003A404001304140023A0840083C70C0092
:106B9000E39E07FC6352400303A404009307000232
:106BA0002300F40003A40400130AFAFF13041400E2
:106BB00023A08400E3160AFE232671016FF09FD7FD
:106BC0002324010093071000930CA000E3CA07E3FD
:106BD0008327C10003A40400938647006FF0DFF50C
:106BE00003C61600930609006FF01FDA83A704009E
:106BF000930650022380D70003A40400130414005A
:106C000023A084006FF01FD3930C00012324010004
:106C10006FF09FDE8327C10003C6160093060900AC
:106C200083A90700938747002326F100E35E0AD477
:106C3000138A09009309F0FF6FF01FD503C61600F1
:106C4000130DD002930609006FF01FD49347FAFF8B
:106C500093D7F74103C61600337AFA00930609006A
:106C60006FF09FD203C61600130D000393060900B0
:106C70006FF09FD183C51600930906FD93060900A6
:106C8000938705FD13860500E3E2FAFA939729003E
:106C9000B38937019386160093991900B389B90017
:106CA00083C50600938909FD938705FD13860500BA
:106CB000E3FEFAFC6FF09FF70327C10083A70400EF
:106CC00083260700130747002326E1002380D7000F
:106CD00003A404001304140023A084006FF09FC5D4
:106CE0009307100063D4070F8327C10093867700B2
:106CF00093F686FF938786002326F10083A946003A
:106D000083A7060063DE090E83A604001306D002E3
:106D1000B307F0402380C60003A40400B336F0009C
:106D2000B30930411304140023A08400138B07001F
:106D3000B389D940930CA000232401006FF05FCEEB
:106D400003C6160013081800930609006FF0DFC38E
:106D500083A70400138908006FF09FE9E3729BCFBB
:106D600093071000930B000093061000E3C447D371
:106D70006FF05FD4979C0100938CCC6493850900DD
:106D800013850C00EF005075330AAA40635240038C
:106D900003A404002300A40103A40400130AFAFFBF
:106DA0001304140023A08400E3160AFE130A000053
:106DB00083C70C00E38207E0E3CC09DA9389F9FF8B
:106DC0001307F0FFE396E9DA6FF0DFDC8327C100F9
:106DD0009386470083A707002326D10093D9F74164
:106DE0006FF05FF2635640019307D002E314FDF8A1
:106DF000979C0100938C0C5D930780026FF01FD766
:106E0000138B0700930CA0002324010003A40400AB
:106E10006FF01FC1130101EB232E3113B70900409E
:106E20009387F9FF2324811423229114232C4113E7
:106E3000232A5113232611142320211523286113FB
:106E40002326711323248113232291132320A113BA
:106E5000232EB111130A05002324B1001794010059
:106E600013040467973A0300938ACA8D979401002C
:106E70009384C42E2326F100930550021305A0002D
:106E800013080004B70610F083470A00638EB704A6
:106E90006388070A03270400130A1A001306170061
:106EA0003387EA009798010023A4C8622300F70003
:106EB0006380A708E31A06FD1737030013078788C6
:106EC000130717008347F7FF23A0F6F0832704007A
:106ED0009387F7FF17960100232CF65EE39207FED7
:106EE00083470A00E396B7FA83461A0013051A008F
:106EF00013070500930B0002130BF0FF130CF0FFB8
:106F00001308000093055005930890009387D6FD61
:106F100093F7F70F130A170063ECF54493972700D4
:106F2000B387970083A70700B387970067800700A0
:106F30001737030013070781E31406F86FF0DFF437
:106F40008320C114032481148324411403290114D0
:106F50008329C113032A8113832A4113032B0113AD
:106F6000832BC112032C8112832C4112032D011299
:106F7000832DC1111301011567800000930C80005F
:106F8000130D00009307100063DA072183278100A7
:106F90009387770093F787FF83AD070003AB470024
:106FA000138787002324E10013860C00930600005A
:106FB00013850D0093050B00EF10005D2328A10041
:106FC00063086D45130941019309100013860C00F5
:106FD0009306000013850D0093050B00EF1080173A
:106FE00013860C0093060000930D0500138B05001B
:106FF000EF1080592320A900938919001309490033
:10700000E3166DFDE3F49DFD13060004B70610F0D2
:1070100063D489038327040013871700B387FA001A
:107020009795010023A6E54A23807701630AC706E6
:10703000130CFCFFE3C089FF8327C1001305C100C7
:1070400093089000B386F9009396260093070101F8
:10705000B386D7001308A00013030004370610F00E
:10706000E38CA6E083A706009305000363F4F80011
:107070009305700503270400B387B7009305170035
:107080003387EA00179E01002324BE442300F70043
:1070900063860737638C65329386C6FF6FF05FFCAB
:1070A000172703001307076A130717008347F7FF23
:1070B00023A0F6F0832704009387F7FF979501003C
:1070C00023A8F540E39207FE130CFCFF6FF09FF638
:1070D0008327040013060004138717009795010007
:1070E00023A8E53EB386FA00930500032380B6008B
:1070F0006308C750938727009796010023AAF63CA0
:107100003387EA00930680072300D7001727030080
:1071100013074763B70610F06392C70213071700FF
:107120008347F7FF23A0F6F0832704009387F7FF38
:1071300017960100232EF638E39207FE832781007D
:10714000930C0001130D0000938747000327810073
:10715000130B0000832D07002324F1006FF0DFE400
:107160008327810083AC070013894700638E0C4C92
:107170006358802B9307D0026394FB3E03C70C0037
:10718000930507006314072A6F00002F9307100070
:10719000930CA000130D0000E3CA07DF83278100D2
:1071A000938747006FF09FFA83278100834617007B
:1071B00013070A0003AB0700938747002324F1005D
:1071C000E3560CD4130C0B00130BF0FF6FF01FD41D
:1071D00083461700930BD00213070A006FF01FD3EA
:1071E0009347FCFF93D7F74183461700337CFC009D
:1071F00013070A006FF09FD183461700930B00031B
:1072000013070A006FF09FD003461700138B06FD8B
:1072100013070A00930706FD93060600E3E2F8FA57
:1072200093172B00B3876701130717009397170075
:10723000B387C70003460700138B07FD930706FDBE
:1072400093060600E3FEF8FC6FF09FF783258100AC
:10725000832704001306A00003A7050093861700E8
:10726000B387FA00179501002324D5262380E70071
:10727000138945006300C736930700046384F62A28
:10728000232421016FF05FBF9307100063DE0735F1
:107290008327810013877700137787FF9307870081
:1072A0002324F100032B47008327070063560B3E7E
:1072B00003270400130600049306170097950100A6
:1072C00023A8D5203387EA009305D0022300B70016
:1072D000638CC638B307F0403337F000330B60419E
:1072E000938D0700330BEB40930CA000130D0000AF
:1072F0006FF09FCB834617001308180013070A008E
:107300006FF0DFC08346170013070A006FF01FC03D
:1073100083270400930600041387170017960100C3
:107320002328E61AB387FA00130650022380C70009
:10733000E314D7B4172703001307C740B70610F0AC
:10734000130717008347F7FF23A0F6F083270400F5
:107350009387F7FF17960100232CF616E39207FE9A
:107360006FF09FB1930C0001130D00006FF09FC1EF
:107370008327040093060004130A050013871700EF
:10738000179601002326E614B387FA00130650026D
:107390002380C700E312D7AE172703001307873AED
:1073A000B70610F0130717008347F7FF23A0F6F086
:1073B000832704009387F7FF17960100232AF6100E
:1073C000E39207FE130A05006FF01FAB17270300B7
:1073D00013074737130717008347F7FF2320F6F0FB
:1073E000832704009387F7FF9795010023A2F50EEA
:1073F000E39207FE9386C6FF6FF09FC61727030030
:1074000013074734E39805FC9386C6FF6FF05FC50A
:10741000E3FA9DBB930910006FF01FBF130C00002F
:1074200003C70C0093050700E30C07E49308F0FF83
:107430001305A00013080004B70610F0635E0B0CE0
:107440008327040013861700B387FA0017930100FF
:107450002320C3082380E7006382A5086308060B86
:10746000938C1C0003C70C00130CFCFF9305070052
:10747000E31607FCE35680E183270400930500022E
:1074800013060004B70610F06F00C000130CFCFFD9
:10749000E3080CDE13871700B387FA002380B700D8
:1074A000179501002326E50293070700E310C7FEA6
:1074B0001727030013070729130717008347F7FF50
:1074C00023A0F6F0832704009387F7FF17950100A8
:1074D0002320F500E39207FE6FF05FFB1727030000
:1074E00013074726E30E06F6130717008347F7FF37
:1074F00023A0F6F0832704009387F7FF1796010077
:107500002328F6FCE39207FE6FF09FF51727030090
:10751000130747236FF05FFD130BFBFFE3121BF311
:107520006FF05FF5172703001307C721B70610F0A8
:10753000130717008347F7FF23A0F6F08327040003
:107540009387F7FF179601002324F6F8E39207FECE
:10755000232421016FF05F92979C0100938C8CE6AD
:1075600093050B0013850C00EF000077330CAC4043
:10757000E35880EB8327040013060004B70610F0DD
:107580006F00C000130CFCFFE30A0CE81387170020
:10759000B387FA00238077019795010023AAE5F2CB
:1075A00093070700E310C7FE172703001307871987
:1075B000130717008347F7FF23A0F6F08327040083
:1075C0009387F7FF9795010023A4F5F0E39207FE58
:1075D0006FF05FFB172703001307C716E39806F445
:1075E000232421016FF05F898327810013874700DF
:1075F00083A707002324E10013DBF7416FF01FCBC3
:107600001727030013070714B70610F01307170016
:107610008347F7FF23A0F6F0832704009387F7FF43
:10762000179601002326F6EAE39207FE930710005F
:1076300017970100232EF7E8930780071727030009
:107640002302F7106FF09FAF635680019307D002BB
:10765000E394FBF0979C0100938CCCD61307800237
:10766000930580026FF09FDC972603009386860DBA
:10767000370610F09386160003C7F6FF2320E6F0C6
:10768000032704001307F7FF9795010023A2E5E401
:10769000E31207FE6FF01FC4938D0700930CA00048
:1076A000130D00006FF05F90B70710F023A0A7F252
:1076B0006F000000130101FC130341022322B102F9
:1076C00093050300232E11002324C1022326D10297
:1076D0002328E102232AF102232C0103232E110384
:1076E00023266100EFF00FF38320C1011305000092
:1076F0001301010467800000130101FB13038103E0
:10770000232481022326A100232CC1021304050097
:10771000130603001305C100232611022322F104DE
:10772000232ED1022320E104232401052326110561
:10773000232E6100EFF04F9B8327C10023800700B9
:107740000325C1008320C102330585400324810243
:107750001301010567800000B70710F083A647F406
:1077600003A607F403A747F4E31AD7FEB7160000F1
:10777000938606FAB306D60033B6C600B305E60014
:1077800023A4D7F423A6B7F467800000B70710F04E
:1077900003A747F403A607F483A647F4E31AD7FE2A
:1077A000B7160000938606FAB306D60033B6C600B5
:1077B00023A4D7F4B305E60023A6B7F49307000883
:1077C00073A0473067800000130101FF232481006C
:1077D0002326110097970100938707D01794010083
:1077E000130444CF03A70700832704001306F07C8B
:1077F00093064706938747069795010023AED5CC9D
:107800009795010023A8F5CC634AD6008320C100D8
:1078100003248100130101016780000013074789D9
:107820009797010023AAE7CAEF00C0499307100009
:107830006316F50203270400B71700009387F77655
:1078400013050000E3D4E7FCEFF01FE603248100FA
:107850008320C100130101016FB05FB817950100CB
:107860001305C5B6EFF01FE513052000EFF0DFE3C9
:10787000032481008320C100130101016FB01FB6F2
:1078800017950100130505B66FF0DFE217950100AB
:107890001305C5B56FF01FE2130101FF232481001A
:1078A0002322910023261100B71400001794010031
:1078B000130444B493878438130000009387F7FFC0
:1078C000E39C07FE13050400EFF0DFDE6FF09FFE80
:1078D0006F008022130101FF23261100EF00803E7C
:1078E0001307100093070000631AE5008320C1000E
:1078F000138507001301010167800000179501003F
:107900001305C5ACEFF01FDB8320C10093072000F7
:1079100013850700130101016780000073700430B4
:107920006F00000067800000737004306F0000007B
:10793000130101FE232A9100232E1100232C810024
:107940002328210123263101835745031307901D66
:10795000930405006382E70E636EF70A6384070CE5
:107960001307801D639AE7081394250097290300E5
:10797000938949E133898900032509011306000031
:1079800093050900EFA00FF09307B0FF6304F5140F
:10799000930710006306F500179701002324F7B43E
:1079A000B387890003A507021306000093050900A9
:1079B000EFA0CFDA9307C0FF6306F50A9307B0FF85
:1079C0006308F50E930710006306F5001797010092
:1079D000232AF7B0B387890003A507011306F0FF38
:1079E00093050900EFA00FEA9307C0FFE31EF5F827
:1079F0009307801D239AF4028320C101032481018F
:107A000083244101032901018329C10013010102DB
:107A1000678000001307E01E6388E7061307F01E67
:107A2000E39CE7FC972903009389C9D513942500AB
:107A3000338989006FF01FFA1394250097290300FA
:107A4000938949D4B387890003A507023389890044
:107A50001306000093050900EFA04FD09307C0FF65
:107A6000E31EF5F49307E01E239AF4028320C1017C
:107A70000324810183244101032901018329C100D9
:107A80001301010267800000139425009729030069
:107A9000938949CF33898900032509021306000021
:107AA00093050900EFA08FCB9307B0FFE31CF5F01F
:107AB0009307F01E239AF4028320C101032481015D
:107AC00083244101032901018329C100130101021B
:107AD000678000009307901D239AF4028320C10160
:107AE0000324810183244101032901018329C10069
:107AF0001301010267800000130101FD23248102AC
:107B00002322910223202103232E31012326110257
:107B100023260100972403009384C4C81729030077
:107B2000130949C71304000097090000938989E0ED
:107B3000130600009305400013051000EF900FC2DC
:107B400023A0A400130600009305400013051000B5
:107B5000EF90CFC02320A90003A5040093060000E6
:107B60009305C10013060000EF904FD313060400E5
:107B70009305100013850900EF805FBB1304140008
:107B8000930740009384440013094900E312F4FA78
:107B90008320C102032481028324410203290102BC
:107BA0008329C10113010103678000009797010039
:107BB0009387079383A707001307301F9387170046
:107BC000637CF70E130101FD232021031729030015
:107BD000130949BD2324810223229102232E31015E
:107BE000232C4101232611029797010023AA078E17
:107BF00013040900972903009389C9BB179A010050
:107C0000130ACA8D93041000032504001306C10053
:107C10009305810023260100EFA0CFDE630E9506B9
:107C20009797010023A0978C13044400E31E34FDB2
:107C300083270A00172403001304C4B59799010091
:107C40009389C98993871700179701002328F7881C
:107C50009304100003250400130600009385090017
:107C6000EFA08FCF1304440063069500979701009F
:107C700023AA9786E31089FE8320C1020324810290
:107C800083244102032901028329C101032A8101BE
:107C900013010103678000000327810083270A0086
:107CA0006306F7009797010023AE97828327C100F0
:107CB000E39807F66FF05FF7179701002322F7822A
:107CC00067800000979701009387C78103A507008D
:107CD0001335150067800000B305B5009307050054
:107CE0006386B70003C70700631607003385A74004
:107CF00067800000938717006FF09FFE93080000D5
:107D000063DC05003305A040B337A000B305B040E5
:107D1000B385F5409308F0FF63DA06003306C040F0
:107D2000B337C000B306D040B386F6401308060050
:107D30001383060093070500138705006398062444
:107D4000978601009386065763F8C50E370E01002B
:107D5000637AC60D130EF00F6374CE001303800018
:107D6000335E6600B386C60103CE0600330E6E0096
:107D7000130300023303C341630C0300B395650092
:107D8000335EC501331866003367BE00B317650064
:107D9000135E0801B355C7031315080113550501F8
:107DA00093D607013376C703B305B5021316060150
:107DB000B366D60063FAB600B386060163E6060131
:107DC00063F4B600B3860601B386B64033F7C60344
:107DD0009397070193D70701B3D6C603B306D5021D
:107DE00013150701B367F50063FAD700B3870701DE
:107DF00063E6070163F4D700B3870701B387D74071
:107E000033D5670093050000638C0800B307A040DA
:107E10003337F000B305B04013850700B385E54064
:107E200067800000370E000113030001E36AC6F308
:107E3000130380016FF0DFF26316060013081000D1
:107E400033586802370701006372E80A1307F00F1E
:107E5000637407011303800033576800B386E6009C
:107E600003C6060033066600130300023303C34053
:107E700063180308B38505419356080113150801DB
:107E80001355050113D6070133F7D502B3D5D50233
:107E9000131707013367C700B305B502637AB7004C
:107EA00033070701636607016374B70033070701EF
:107EB000B305B74033F7D5029397070193D707016E
:107EC000B3D5D502B305B50213150701B367F500A5
:107ED00063FAB700B387070163E6070163F4B700ED
:107EE000B3870701B387B7406FF09FF137070001F1
:107EF00013030001E362E8F6130380016FF0DFF57E
:107F00003318680033DEC500935E08013356C500A0
:107F1000B31765003355DE03B39565003366B600CD
:107F20009315080193D50501935606013377DE03B7
:107F30003385A502131707013367D700637AA700BB
:107F400033070701636607016374A700330707015E
:107F5000B306A74033F7D6031316060113560601DE
:107F6000B3D6D60313170701B386D502B365C7008E
:107F700063FAD500B385050163E6050163F4D50016
:107F8000B3850501B385D5406FF01FEFE3EED5E66D
:107F90003708010063FC0605930EF00F33B8DE00CE
:107FA0001318380033DE06011783010013038330F2
:107FB0003303C301834E0300130E0002B38E0E0180
:107FC000330EDE41631E0E0263E4B600636AC50031
:107FD000B307C540B385D5403335F5003387A54099
:107FE00013850700930507006FF01FE237030001B8
:107FF00013080001E3E866FA130880016FF09FFAA6
:108000003357D601B396C601B366D700B357D5012F
:1080100033D7D501B395C501B3E7B70093D50601B2
:108020003373B702139F0601135F0F0113D80701C3
:108030003316C6013315C5013357B70213130301B5
:1080400033680301B30FEF0213030700637EF801E7
:108050003308D8001303F7FF6368D8006376F8018C
:108060001303E7FF3308D8003308F841B37FB802A1
:108070003358B802939F0F01B3050F03139F0701F5
:10808000135F0F0133EFEF0113070800637EBF009A
:10809000330FDF001307F8FF6368DF006376BF006C
:1080A0001307E8FF330FDF0013130301B70F0100BD
:1080B0003363E3009387FFFF13580601330FBF407C
:1080C000B375F30013530301B377F6003387F5025A
:1080D000B307F302B385050333030303B385F50048
:1080E000135807013308B8006374F8003303F30131
:1080F000B70701009387F7FF935508013378F8001D
:10810000131808013377F700B38565003307E800DB
:108110006366BF00631EBF00637CE5003306C74093
:108120003337C700B385D540B385E5401307060054
:108130003307E5403335E500B305BF40B385A540BF
:10814000B397D5013357C70133E5E700B3D5C50170
:108150006FF09FCB93870500130806001387060076
:1081600013030500639606289788010093888814F6
:1081700063F6C50E370701006378E60C1307F00FAE
:108180003337C70013173700B356E600B388D8005B
:1081900083C608003387E60093060002B386E640F4
:1081A000638C0600B397D7003357E5003318D60029
:1081B000B365F7003313D50013550801B3D7A502F3
:1081C00013160801135606019356030133F7A5024F
:1081D000B305F60213170701B366D700138707002C
:1081E00063FEB600B38606011387F7FF63E8060156
:1081F00063F6B6001387E7FFB3860601B386B64081
:10820000B3F7A6021313030113530301B3D6A60257
:108210009397070133E36700B305D6021385060081
:10822000637CB300330368001385F6FF63660301C4
:108230006374B3001385E6FF131707013367A700C4
:10824000930500006F00400EB70600011307000100
:10825000E36CD6F2130780016FF01FF3631606007C
:108260009306100033D8C602B70601006372D80C1B
:108270009306F00F63F4060113078000B356E8007D
:10828000B388D80083C60800B386E600130700024F
:108290003307D7406318070AB387074193051000D7
:1082A000135608019318080193D808019356030147
:1082B00033F7C702B3D7C70213170701B366D70056
:1082C0003385F8021387070063FEA600B386060114
:1082D0001387F7FF63E8060163F6A6001387E7FF3D
:1082E000B3860601B386A640B3F7C6021313030193
:1082F00013530301B3D6C6029397070133E3670014
:10830000B388D80213850600637C13013303680029
:108310001385F6FF63660301637413011385E6FF9B
:10832000131707013367A7001305070067800000D4
:10833000B706000113070001E362D8F413078001B8
:108340006FF0DFF33318E800B3D5D7003313E5003F
:10835000B356D50013550801B397E70033F7A502CC
:10836000B3E8F6009317080193D7070113D6080165
:10837000B3D5A502131707013367C700B386B70249
:1083800013860500637ED700330707011386F5FFC8
:10839000636807016376D7001386E5FF330707019B
:1083A000B306D74033F7A6029398080193D8080183
:1083B000B3D6A60213170701B385D702B367170117
:1083C0001387060063FEB700B38707011387F6FF24
:1083D00063E8070163F6B7001387E6FFB387070179
:1083E000B387B74093150601B3E5E5006FF05FEB87
:1083F00063E6D5183707010063F4E6041308F00FAD
:108400003337D8001317370033D8E60097850100BB
:10841000938545EAB385050103C80500930500026D
:108420003308E800B3850541639605021307100081
:10843000E3ECF6EE3335C500134715006FF0DFEEC1
:10844000B705000113070001E3E0B6FC1307800144
:108450006FF09FFB33570601B396B600B366D700A3
:1084600093DE060133D70701B378D703B397B7007C
:10847000335805013363F8009397060193D707013A
:10848000135803013316B6003357D70393980801E6
:1084900033E80801338FE702130E0700637EE8011B
:1084A0003308D800130EF7FF6368D8006376E8013D
:1084B000130EE7FF3308D8003308E841B378D80338
:1084C0003358D80393980801B38E07039317030119
:1084D00093D70701B3E7F8001307080063FED7013D
:1084E000B387D7001307F8FF63E8D70063F6D70117
:1084F0001307E8FFB387D700131E0E01B387D741D8
:10850000B70E01003367EE001388FEFF33730701D7
:10851000935807013378060113560601330E0303FF
:108520003388080393560E013303C3023303030158
:10853000B3866600B388C80263F40601B388D80125
:1085400013D60601B308160163E61703E39A17CFA3
:10855000B70701009387F7FFB3F6F600939606017D
:10856000337EFE003315B500B386C60193050000C7
:10857000E37CD5DA1307F7FF6FF09FCC930500007B
:10858000130700006FF05FDA9308060013870600F8
:108590009307050013880500639C06229786010057
:1085A000938646D163FCC50C37030100637E660ADF
:1085B0001303F00F6374C300130780003353E60006
:1085C000B386660003CE060013030002330EEE00EE
:1085D0003303C341630C0300B3956500335EC501EB
:1085E000B31866003368BE00B317650013D60801E0
:1085F0003377C802139508011355050193D6070177
:108600003358C80213170701B366D70033080503B0
:1086100063FA0601B386160163E6160163F40601E8
:10862000B3861601B386064133F7C6029397070156
:1086300093D70701B3D6C602B306D50213150701B7
:10864000B367F50063FAD700B387170163E6170134
:1086500063F4D700B3871701B387D74033D56700DA
:108660009305000067800000370300011307000135
:10867000E36666F4130780016FF05FF4631606008B
:1086800013061000B35816033706010063F2C80A38
:108690001306F00F637416011307800033D6E80049
:1086A000B386C60003CE060013030002330EEE00AD
:1086B0003303C34163180308B385154113D7080179
:1086C000139508011355050113D60701B3F6E5020A
:1086D000B3D5E50293960601B3E6C600B305B5022D
:1086E00063FAB600B386160163E6160163F4B600BA
:1086F000B3861601B385B640B3F6E502939707013A
:1087000093D70701B3D5E502B305B502139506016A
:10871000B367F50063FAB700B387170163E6170183
:1087200063F4B700B3871701B387B7406FF01FF347
:108730003706000113070001E3E2C8F613078001C2
:108740006FF0DFF5B398680033D7C501B317650044
:10875000335EC50113D50801B376A702B395650052
:10876000336EBE009395080193D5050113560E0193
:108770003357A70293960601B3E6C6003387E50296
:1087800063FAE600B386160163E6160163F4E600B9
:10879000B38616013386E640B376A602131E0E0199
:1087A000135E0E013356A602939606013386C50268
:1087B000B3E5C60163FAC500B385150163E615018B
:1087C00063F4C500B3851501B385C5406FF01FEF95
:1087D000E3EAD5E83707010063FCE604930EF00FE7
:1087E00033B7DE001317370033D3E6009788010054
:1087F000938848ACB388680083CE0800130E00024B
:10880000B38EEE00330EDE41631E0E0263E4B6004B
:10881000636AC500B307C540B385D5403335F5005D
:108820003388A54013850700930508006FF09FE388
:10883000B708000113070001E3E816FB13078001E6
:108840006FF09FFA3357D601B396C601B366D700CF
:10885000B357D50133D7D501B395C501B3E7B700F9
:1088600093D506013373B702139F0601135F0F01FF
:1088700093D807013316C6013315C5013357B70224
:1088800013130301B36813013308EF021303070046
:1088900063FE0801B388D8001303F7FF63E8D8002C
:1088A00063F608011303E7FFB388D800B3880841D3
:1088B000B3FFB802B3D8B802939F0F01B3051F03EB
:1088C000139F0701135F0F0133EFEF0113870800B8
:1088D000637EBF00330FDF001387F8FF6368DF009C
:1088E0006376BF001387E8FF330FDF001313030124
:1088F000B70801003363E3009387F8FF13580601BC
:10890000330FBF40B375F30013530301B377F60081
:108910003387F502B307F302B3850503330303037B
:10892000B385F500135807013308B8006374F800E5
:1089300033031301B70701009387F7FF935508012D
:108940003378F800131808013377F700B385650012
:108950003307E8006366BF00631EBF00637CE50069
:108960003306C7403337C700B385D540B385E540EC
:10897000130706003307E5403335E500B305BF4074
:10898000B385A540B397D5013357C70133E5E70059
:10899000B3D5C5016FF01FCD978701009387C7B08E
:1089A00083A60700178701001307C7AE0327070038
:1089B00023A2A600637EE50017870100130747AED8
:1089C0000325070083A50700938545006F800FB23C
:1089D000130101FF232481002326110017870100C2
:1089E000130747AC130405000325070083A5070000
:1089F00093854500EF808FAF978701009387C7A7C6
:108A000083A707006376F4009787010023A687A653
:108A10008320C1000324810013010101678000004D
:108A200097870100938747A803A7070083A607003D
:108A3000832747049387F7FF2322F70483A746047D
:108A4000639407007360043067800000130101FE27
:108A5000232C8100232A9100130405009384050030
:108A600023282101232631012324410123225101FE
:108A7000232E1100EFA09F978327040003290401F0
:108A8000B7090001B3E59700930AC4002320B4009E
:108A9000930400009389F9FF370A000203270400BA
:108AA00063822A050326090013050900B3654701FF
:108AB000B37636019317560033F7E60003294900D1
:108AC00063C60700631607006FF05FFDE398E6FCDE
:108AD0009317760063D40700B3E4D400EFB05FD8F7
:108AE0006FF0DFFB93C4F4FFB3F4E40023209400A1
:108AF000EFA05FC3032504008320C101032481018B
:108B000083244101032901018329C100032A810033
:108B1000832A41001301010267800000130101FF55
:108B20002326110023248100EFE01FFD17F7FFFF2C
:108B30001307C7C9930600001306100093054006EB
:108B4000178501001305858BEFD0CF8763020502DF
:108B500013040500EFA01F8B130605001307000088
:108B6000930600009305100013050400EFD08F97C3
:108B7000EFA00FD58320C10003248100130500005E
:088B80001301010167800000F0
:02000004800278
:10000000E06BFEFF506DFEFFEC6BFEFF506DFEFFE0
:10001000506DFEFF506DFEFF506DFEFF146CFEFF35
:10002000506DFEFF506DFEFF3C6CFEFF4C6CFEFF02
:10003000506DFEFF646CFEFF746CFEFF746CFEFF7F
:10004000746CFEFF746CFEFF746CFEFF746CFEFF3C
:10005000746CFEFF746CFEFF746CFEFF506DFEFF4F
:10006000506DFEFF506DFEFF506DFEFF506DFEFFA8
:10007000506DFEFF506DFEFF506DFEFF506DFEFF98
:10008000506DFEFF506DFEFF506DFEFF506DFEFF88
:10009000506DFEFF506DFEFF506DFEFF506DFEFF78
:1000A000506DFEFF506DFEFF506DFEFF506DFEFF68
:1000B000506DFEFF506DFEFF506DFEFF506DFEFF58
:1000C000506DFEFF506DFEFF506DFEFF506DFEFF48
:1000D000506DFEFF506DFEFF506DFEFF506DFEFF38
:1000E000506DFEFF506DFEFF506DFEFF506DFEFF28
:1000F000506DFEFF506DFEFF506DFEFF506DFEFF18
:10010000B86CFEFFE06CFEFF506DFEFF506DFEFF11
:10011000506DFEFF506DFEFF506DFEFF506DFEFFF7
:10012000506DFEFF406DFEFF506DFEFF506DFEFFF7
:10013000F069FEFFF86AFEFF506DFEFF506DFEFF96
:10014000486BFEFF506DFEFFC06BFEFF506DFEFF63
:10015000506DFEFF086CFEFFAC71FEFF1872FEFFD3
:10016000B871FEFF1872FEFF1872FEFF1872FEFFD4
:100170001872FEFF5070FEFF1872FEFF1872FEFF2D
:100180007870FEFF8870FEFF1872FEFFA070FEFF01
:10019000B070FEFFB070FEFFB070FEFFB070FEFFEB
:1001A000B070FEFFB070FEFFB070FEFFB070FEFFDB
:1001B000B070FEFF1872FEFF1872FEFF1872FEFF8D
:1001C0001872FEFF1872FEFF1872FEFF1872FEFF13
:1001D0001872FEFF1872FEFF1872FEFF1872FEFF03
:1001E0001872FEFF1872FEFF1872FEFF1872FEFFF3
:1001F0001872FEFF1872FEFF1872FEFF1872FEFFE3
:100200001872FEFF1872FEFF1872FEFF1872FEFFD2
:100210001872FEFF1872FEFF1872FEFF1872FEFFC2
:100220001872FEFF1872FEFF1872FEFF1872FEFFB2
:100230001872FEFF1872FEFF1872FEFF1872FEFFA2
:100240001872FEFF1872FEFF1872FEFF1872FEFF92
:100250001872FEFF1872FEFFF470FEFF3071FEFF91
:100260001872FEFF1872FEFF1872FEFF1872FEFF72
:100270001872FEFF1872FEFF1872FEFF9C71FEFFDF
:100280001872FEFF1872FEFF246EFEFF786FFEFFED
:100290001872FEFF1872FEFF0870FEFF1872FEFF54
:1002A0003470FEFF1872FEFF1872FEFF0C72FEFF24
:1002B000000102020303030304040404040404040D
:1002C00005050505050505050505050505050505DE
:1002D00006060606060606060606060606060606BE
:1002E00006060606060606060606060606060606AE
:1002F000070707070707070707070707070707078E
:10030000070707070707070707070707070707077D
:10031000070707070707070707070707070707076D
:10032000070707070707070707070707070707075D
:10033000080808080808080808080808080808083D
:10034000080808080808080808080808080808082D
:10035000080808080808080808080808080808081D
:10036000080808080808080808080808080808080D
:1003700008080808080808080808080808080808FD
:1003800008080808080808080808080808080808ED
:1003900008080808080808080808080808080808DD
:1003A00008080808080808080808080808080808CD
:1003B000546D725100000000546D7220537663003A
:1003C000286E756C6C2900004572726F7220696E20
:1003D00020787878207461736B73200D0A00000018
:1003E0006D69616F750A00006D69616F75320A0091
:1003F00068756E6772790A00436865636B54696D4E
:040400006572000021
:100404001000000000000000017A5200017C01018C
:100414001B0D02001000000018000000DC78FEFF35
:100424005804000000000000100000002C00000030
:10043400207DFEFF340400000000000010000000D6
:10044400400000004081FEFF100400000000000096
:0804E400FC8F0100090000007B
:040000058000004037
:00000001FF
